:020000040800F2
:104000000050002005D1000885A6000887A60008FA
:1040100089A600088BA600088DA6000800000000F5
:1040200000000000000000000000000091A6000851
:104030008FA600080000000093A60008498A000827
:1040400095A6000897A6000899A600089BA6000858
:104050009DA600089FA60008A1A60008A3A6000828
:10406000A5A60008A7A60008A9A600080000000051
:104070000000000000000000000000000000000040
:104080000000000000000000B9A60008BBA6000860
:10409000C5A60008D1A60008DDA60008E9A600080C
:1040A000EBA60008EDA60008EFA60008F1A60008A0
:1040B000F3A60008F5A60008F7A60008F9A6000870
:1040C000FBA60008FDA60008FFA6000801A700083F
:1040D00003A70008BD82000807A7000809A7000879
:1040E0000BA700080DA700080FA70008000000009C
:1040F00000000000000000000000000000000000C0
:0C41000000000000000000005FF800005C
:1041100030BF704720BF704740BF7047BFF36F8FFD
:104120007047BFF34F8F7047BFF35F8F704701DF5A
:104130007047EFF31480704780F31488BFF36F8FDC
:104140007047EFF30980704780F309887047EFF3F9
:104150000880704780F30888704772B6704762B66F
:10416000704771B6704761B6704780F31188704729
:10417000EFF31280704740BA704700BA70470000F2
:104180000C4B10B59B680C4C13F480530B480C4936
:104190000C4A07D0012323700B4B03600B480860C7
:1041A000136010BD23700A4B03600A4B0B600A4B6F
:1041B000F6E700BF000C0140A80E0020B40E00205E
:1041C000080F0020BC0E0020358A0008CF8F0008A1
:1041D0009185000839840008E5840008000000008B
:1041E0002DE9F3410121484807F09EFB01210420FD
:1041F00007F082FE032510264AF21003434C01A962
:104200002046ADF804308DF807608DF8065007F0B1
:10421000F8FA4FF420434FF0040826616361062347
:104220000DEB08012046ADF804308DF807808DF8BD
:10423000065007F0E6FA0121082007F05DFE40F67F
:10424000FC43334F0DEB08013846ADF804308DF8D0
:1042500007608DF8065007F0D4FA40F618433B612A
:10426000E4237B614FF480530DEB08018DF8078048
:104270004FF440483846ADF8043007F580678DF8B4
:10428000065007F0BEFA3046012107F035FE01A9BD
:1042900038468DF80760ADF804808DF806504FF46D
:1042A000005607F0AEFA4823C7F8148001A9384633
:1042B0008DF80730ADF804608DF8065007F0A1FACC
:1042C0000121144807F030FB00230A211A466661D9
:1042D000A06826614504A06858BF0132400448BF69
:1042E00001330139F3D10A2A0B4A0AD10A2B08D12A
:1042F000012301210448137007F016FB02B0BDE84A
:10430000F0810023F5E700BF000230000008014003
:10431000000C014000043000B90E0020F7B5114B2D
:104320001B78E3B14FF400610F4B0F464FF48060F0
:1043300000241E460D4D5F6118610194019AAA4246
:1043400009D9316170610194019AAA42F3D8019AA6
:1043500001320192F8E7019A01320192EEE703B0CF
:10436000F0BD00BFB90E0020000C01403F0D03005E
:1043700010B90422014B5A61704700BF000C014084
:1043800010B90422014B1A61704700BF000C0140B4
:1043900010B50021044644FA01F3DB07C8B205D585
:1043A000FFF7EEFF01310829F5D110BDFFF7E0FF5F
:1043B000F8E7012808B50ED003D3022810D000205A
:1043C00008BD002004F034FC40F24C43984294BFF6
:1043D0000020012008BD054B9868C0F3800008BD8F
:1043E000024B9868C0F3400008BD00BF00080140C0
:1043F00020B9034BD868C0F3800070470020704795
:10440000000C014070B5002401262546E0B2FFF7FC
:10441000D0FF18B106FA04F31D43EDB20134082CA5
:10442000F4D1284670BD08B107F0A2BB07F0A8BBC5
:1044300062B6704772B6704708B9014B1870704782
:104440006805002050B9064B5A6842F040525A6045
:104450004FF400425A610122024B1A70704700BFAC
:1044600000100140680500204022064B10F0010FAB
:1044700014BF5A611A61802210F0020F14BF5A61F2
:104480001A617047000C0140074B9A88C2F307225B
:10449000042A06D19A88D2B2EC2A02D1188980B2B5
:1044A00070470020704700BF006C004038B5174BC4
:1044B000174C9D6815F4005501D0606838BD04F0B4
:1044C0000FFB2A46A060FF21022000F047FB0122DB
:1044D0000546FF21022000F041FB40EA052010F0D4
:1044E000020318BF012380082373C20442BF237B49
:1044F00043F002032373830442BF237B43F004038E
:104500002373236923EA0000606038BD0010014076
:104510006805002038B54C4B9B689B0451D4FFF7CD
:10452000C5FF4A4B5A6990425CDD9969821A8A42FA
:10453000474C0BDA2168D3E908455143641845EB31
:10454000E175996AC3E908450A4449E093F82C10DB
:104550004D0737D51A692468821A5443E517C3E911
:1045600008459A6200240025C3E90C4521F00401A6
:1045700083F82C109A6B9D6AAC1A84EAE471DA6BAA
:10458000A1EBE471914253D99A68196C511A6429CC
:104590004ED91A6442F21072624392FBF1F13C224E
:1045A0004A4319699D63013192FBF1F240F6B8313B
:1045B000002A5A64B8BF52428A4228DDC822DA6310
:1045C000586138BD196901318A1A2168D3E9084553
:1045D0005143641A65EBE175C3E90845996A8A1A83
:1045E0009A62C7E7C6DA9969121A8A42184CECDB5C
:1045F00093F82C104D0706D5246898624443E517BC
:10460000C3E90845AEE7196901318A1A92E7B2F5A4
:104610007A7F01DD6422D2E7322A01DD0A22CEE769
:104620000A2A01DD0522CAE7012AC9DD0122C6E7FF
:104630009A68196C521AB2F5FA6F81BF0122DA63D7
:1046400000225A64BCE700BF00100140680500204A
:104650000400002008B568B9FFF75CFF0649D1E9FE
:104660000823D1E90C01121A63EB0103100A40EA96
:10467000036008BD002008BD6805002038B50D4660
:10468000E0B9114CFFF746FFD4E908012269002880
:1046900071F100034FEA02224FEAE2730FDB0AF0E6
:1046A0002FFDC4E90C23E9170B022A02D4E90C01FF
:1046B00043EA156312184B41C4E9082338BD404250
:1046C00061EB4101EBE700BF6805002010B9024B28
:1046D00009011960704700BF0400002010B9024BA7
:1046E00083F82C10704700BF68050020014B586C00
:1046F000704700BF6805002010B9024B187B704757
:10470000002070476805002010B50022FE2102201D
:1047100000F024FA01224021022000F01FFA0022BA
:104720000220114600F01AFA04460122002102205C
:1047300000F014FA082C0CBF40F6FF7340F2FF3370
:104740000E4C4FF000020BBF236123614FF4006356
:104750004FF40073E7210220A36100F0FFF900216C
:104760000122022000F0FAF9FFF7A0FE60610002CA
:10477000C117C4E90C01C4E9080110BD6805002097
:1047800008B5082004F054FA77281BD9184B93F881
:10479000482012B9012283F84820082004F048FA82
:1047A000772817D9124B1B78A3B903F1804303F57F
:1047B00088335A6822F030425A605A6842F0804288
:1047C0005A6008BD082004F033FA6D28E5D80022AD
:1047D000074BE0E7082004F02BFA6D2807D8054BBB
:1047E0005A6842F040525A604FF400425A6108BD84
:1047F0006805002000100140044B93F84800013880
:1048000001288CBF00200120704700BF68050020F0
:10481000044B93F8480001280ABF0222002083F8C5
:10482000482070476805002008B5FFF73FFE0528BF
:1048300008D9FFF73BFE40F2F933984294BF0020BD
:10484000012008BD012008BD37B5144B4FF480424C
:1048500098B95A610623ADF8043003238DF8063069
:10486000042300F180400DEB030100F584308DF846
:10487000073006F0C6FF03B030BD1A6103230225DE
:104880008DF806301023064C01A92046ADF80450DF
:104890008DF8073006F0B5FF6561ECE700100140C8
:1048A0000008014008B540B904F0C2F940F24C4399
:1048B000984294BF0020012008BD002008BD18B90F
:1048C000024B93F82C0070470020704768050020C9
:1048D0004FF480323A21002005F00ABA2DE9F7435F
:1048E000474D044605EB4015AB680BB16E8B96B98E
:1048F0003821204605F026FA382120F4806220462F
:1049000005F0F6F94FF480323A21204603B0BDE8B5
:10491000F04305F0EDB905F0AEFBC0F1080006FA72
:1049200000F009F0E1FDAD68064685EAE570A0EB10
:10493000E5700F4609F0D8FD02460B463046394671
:1049400009F062FF2F4B002206460F4609F032FEA7
:104950006A46804689460AF075FE002200230AF066
:1049600091F8A0B1494640460AF0D4F8002D064619
:104970004FF03801B8BF4642204605F0E3F9382130
:1049800020F48062204605F0B3F93246BCE7304699
:1049900039466A460AF056FE002D06460F46DDE906
:1049A000000118DD0AF0B6F813A3D3E900230504CB
:1049B0003946304609F0FEFD0AF0ACF805433821CF
:1049C000204605F0BFF9382140F48062204605F00A
:1049D0008FF92A4698E70AF09DF807A3D3E9002348
:1049E000C5433946304609F0E5FD0AF093F8C0F5B5
:1049F0001C502D041030E1E7000000000088C34087
:104A0000000A00200000F04010B5044605F033FB1A
:104A1000054BC0F1080053F820102046BDE81040B7
:104A20004909FFF753BE00BF3CFE00082DE9F04FD7
:104A3000012189B04FF4804007F06AFA012108464D
:104A400007F05AFA03264FF420434FF0180A3F4C60
:104A500002A92046ADF808308DF80BA04FF0040BEA
:104A60008DF80A6006F0CDFE4FF4804302A920467F
:104A7000ADF808308DF80A608DF80BB006F0C1FE75
:104A80001023002401254FF482794FF002084FF4DF
:104A90000077ADF818302E4B03A91846ADF80C403E
:104AA000ADF81040ADF81A40ADF81C400193ADF8D8
:104AB0000E90ADF81280ADF81450ADF8167007F0F6
:104AC000D3FA019B2946184607F052FB29464FF4BA
:104AD000805007F011FA2146284606F025FFA02352
:104AE0008DF80BA0DFF870A002A95046ADF8083091
:104AF0008DF80A6006F085FE402302A95046ADF805
:104B000008308DF80A608DF80BB006F07AFE282385
:104B1000ADF80C40ADF81040ADF81A40ADF81C40AF
:104B20000C4C03A92046ADF81830ADF80E90ADF846
:104B30001280ADF81450ADF8167007F095FA2946BA
:104B4000204607F015FB09B0BDE8F08F000C0140CE
:104B50000038004000300140000801400128F8B54D
:104B600005460E4614462BD003D302282AD0002433
:104B700054E010222A4B2B4F5A610221384607F08D
:104B800079FB0028F9D03146264807F01FFB254E57
:104B90000121304607F06EFB0028F9D0002C39D0F7
:104BA000012D35D02CD3022DE1D110221E4B1A61DC
:104BB0001E4A13889BB243F0020313801B4823E074
:104BC0000822D7E71022194D2B8823F002031B047B
:104BD0001B0C2B80144B5A610221284607F04AFB1C
:104BE0000028F9D03146114807F0F0FA0F4D0121A5
:104BF000284607F03FFB0028F9D0002CDED0D4E790
:104C00001022074B1A61074807F0E2FAC4B205E028
:104C10000822F6E7012DF6D9022DCFD02046F8BDA7
:104C2000000C014000380040000801400030014005
:104C3000044B9A78044B12B104221A707047032275
:104C4000FBE700BF280A00209C0A002073B5CB4D6B
:104C5000AE786A782C461EB10422C94B1A70FDE169
:104C6000A52A00F0588300F2C280152A00F046827F
:104C700055D80C2A00F0F4812ED8042A00F0B58112
:104C80000AD8012A00F09381002A00F08781022AC5
:104C900000F091810322E0E7062A00F0C881C0F00D
:104CA000B881072AF6D11021002005F04BF8034601
:104CB000EA78A878D2080192C3F307220092C3F3DE
:104CC00007430022102104F0DFFFAA78AD4B03EB6D
:104CD0004213EA785A77C1E1102A00F0EF810CD82C
:104CE0000E2A00F0DC8140F2CB81A74BD5F80300FF
:104CF0009B6898472421024653E1122A00F0EE8176
:104D0000C0F0E481132A00F0F181142AC2D19E4B35
:104D1000D5F803001B6898472B21024641E1202A61
:104D200000F03E8233D8192A00F00A8212D8172ADE
:104D300000F0FB8140F2E6813421002005F002F80A
:104D4000D5F803300246A878002B00F0F68142F037
:104D5000080290E11B2A00F01182C0F000821C2A98
:104D600000F015821F2A95D11021002004F0EAFFDF
:104D70000246D1B2C2F30722EB78A87801910092E3
:104D80001021002203F00F0304F07EFF66E1A02A49
:104D900000F0A18217D87F2A00F013828C2A00F03D
:104DA0001982212A7FF476AF6E21002004F0CAFF19
:104DB0000246D1B2C2F30722EB78A87801910092A3
:104DC0006E210022E0E7A22A00F09382C0F08A82DE
:104DD000A32A00F09782A42A7FF45CAF0020D5F8C4
:104DE0000310C9B202B0BDE8704005F0B9B8BF2ADF
:104DF00000F0468353D8AE2A00F0E18225D8A92AD4
:104E000000F0B9820DD8A72A00F0AC8240F2978258
:104E10000020D5F80310C9B202B0BDE8704005F01B
:104E2000D5B9AB2A00F0B982C0F0AE82AC2A00F04E
:104E3000BD82AD2A7FF42EAF0020D5F80310C9B291
:104E400002B0BDE8704005F0D3B9B82A00F0DE82A8
:104E500011D8B52A00F0BC82B62A00F0C482B12A6B
:104E60007FF418AF0020D5F80310C9B202B0BDE836
:104E7000704005F01BB8BA2A00F0DA82C0F0CF8289
:104E8000BB2A00F0E882BC2A7FF404AF0020D5F8EA
:104E90000310C9B202B0BDE8704005F048BAD22A8A
:104EA00000F0BC8132D8C32A00F0AA810CD8C12AF4
:104EB00000F0A18140F2ED82334BD5F803001B686E
:104EC0009847304B1860C9E0CA2A00F0A1810FD87A
:104ED000C92A7FF4DFAE3821002004F033FFD5F873
:104EE000033000F4806223F480631A4338219CE08D
:104EF000CC2A00F0D782D12A7FF4CCAE0020D5F89E
:104F0000031002B0BDE87040FFF7B8BBD92A00F02B
:104F1000A0810DD8D62A00F08881D82A00F095818A
:104F2000D42A7FF4B7AED5F80320164BDA6095E0AB
:104F3000FB2A00F0988107D8DA2A7FF4ABAED5F8C7
:104F40000320104B1A6189E0FE2A00F09C81FF2AA1
:104F50007FF4A0AED5F80330002B00F0B381012B15
:104F60007FF47AAE074A5376074B084A1A60084A1C
:104F70001A61084A9A60084AABE100BF280A00207B
:104F80009C0A0020000A0020B4050020B5A50008F6
:104F900019A60008F1A5000859A600082D21D5F88A
:104FA0000320002002B0BDE8704004F0A1BED5F897
:104FB00003202121F5E7D5F803302021002BC8BFBD
:104FC0000122002004F094FE0122AD78B64BD4F803
:104FD00003005A55B54B002853F82530B8BF40425E
:104FE0009847272102462846DCE7D5F80300AF4C56
:104FF0000028B8BF40422368984720216060A87805
:1050000004F0A0FE50BBA878272104EB800462685E
:10501000C8E70022A64BD5F803001A70A34B9B6883
:10502000984726210246A34B1860A078BAE71021C2
:10503000002004F087FE0346DAB2A8780192EA78ED
:10504000C3F30743D20800921021002204F01CFE93
:10505000AA78994B03EB4213EA781A7702B070BD35
:105060003421304604F06EFED5F803300246A878AD
:105070001BB942F00202342194E722F00202FAE75F
:105080003421002004F05EFED5F803300246A878F3
:1050900013B942F00102EEE722F00102EBE73421FE
:1050A000002004F04FFED5F803300246A87813B173
:1050B00042F01002DFE722F01002DCE77B4BD5F86C
:1050C00003001B689847252102466AE7774BD5F80D
:1050D00003009B6898472821024662E7734BD5F886
:1050E00003009B6898472A2102465AE76F4BD5F880
:1050F00003001B6898472321024652E7D5F8032096
:105100002C214EE7D5F803000028FFF6A5AD6A4B29
:105110005B7E012B01D005F07FFA20B1674AB2FB1C
:10512000F0F2152181E7664AFBE7604BD5F80300F2
:105130001B6898473321024633E722F008029AE7BA
:105140003421304604F0FEFDD5F803300246A8783D
:1051500013B142F004028EE722F004028BE73421FF
:10516000002004F0EFFDD5F803300246A87813B113
:1051700042F400627FE722F400627CE70020D5F869
:105180000310C9B202B0BDE8704004F0A1BE002017
:10519000D5F80310C9B202B0BDE8704004F0AABE51
:1051A0006E21304604F0CEFDEB78AC7801932B797C
:1051B000324603F0030300936E21C0F307432046F9
:1051C000E2E5D5F80330022B3FF646ADEA78374BDF
:1051D0001A7343E7D5F803100020C1F10801C9B2E2
:1051E00004F052FEA878FFF779FBA07802B0BDE882
:1051F0007040FFF709BCD5F803202F4B1A762DE736
:105200002A4BD5F803001B6898472B4B586025E7BD
:10521000D5F80320284B00205A83E4E73046E9788C
:1052200002B0BDE87040FFF759BAD5F8030009F0A5
:105230005BF91BA3D3E9002309F0E6FA0AF0F0FAC0
:1052400009F068FC11210246ABE6D5F803203921AC
:10525000A7E63046D5F80320174B9A6002B0BDE8A8
:105260007040FFF73BBB0021084604F06BFDD5F80A
:1052700003100246A87819B122F01002002191E62D
:1052800042F010028EE6D5F80330012B3FF6E4AC75
:10529000E87802B0BDE87040FFF7D6BAAFF30080FF
:1052A0002D431CEBE236FA3FF5090020B40500203F
:1052B000240A0020200A0020000A00200024F40014
:1052C000B50010007C4A53767C4B7D4A1A601A6107
:1052D0009A605A61C2E63046E97802B0BDE8704093
:1052E00004F090BE0020E97802B0BDE8704004F000
:1052F00077BE0020D5F80310C9B202B0BDE87040F7
:1053000004F09EBD0020D5F80310C9B202B0BDE87C
:10531000704004F001BE304604F0C9FED5F8031019
:10532000AB78C9B228B9184602B0BDE8704004F0A5
:1053300055BE184602B0BDE8704004F023BE002000
:1053400004F0B5FED5F80310C9B228B9A87802B0A8
:10535000BDE8704004F062BDA87802B0BDE87040BE
:1053600004F02ABE0020D5F80310C9B202B0BDE88F
:10537000704004F039BD3046D5F80310C9B202B010
:10538000BDE8704004F0DDBE0020D5F80310C9B2BE
:1053900002B0BDE8704004F0E6BE0020D5F803106E
:1053A000C9B202B0BDE8704004F0B9BE0020D5F823
:1053B0000310C9B202B0BDE8704004F0E6BE30464A
:1053C000D5F80310C9B202B0BDE8704004F0EEBEDB
:1053D000D5F803000028FFF63FAC384B1B68984710
:1053E000354B58613AE6D5F803000028FFF634AC97
:1053F000314B5B7E012B01D005F00EF920B1314A13
:10540000B2FBF0F2142110E62F4AFBE73046D5F844
:105410000310C9B202B0BDE8704004F08FBD002097
:10542000D5F80310C9B202B0BDE8704004F01ABD4F
:10543000D5F803000028FFF60FAC1F4B5B7E012B55
:1054400001D005F0E9F820B11E4AB2FBF0F21321B9
:10545000EBE51D4AFBE7D5F803100020C9B204F0C4
:1054600056FF0021A87804F06DFCD5F80310024621
:10547000A87811B142F0040200E722F0040291E59D
:105480003046D5F80310C9B202B0BDE8704004F050
:105490002CBF0020D5F80310C9B202B0BDE870409F
:1054A00004F011BF0020D5F80310C9B202B0BDE866
:1054B000704004F0E4BE00BF000A0020B4050020E4
:1054C00081A600080024F400B500100038B5B34BE5
:1054D0009A781C46022A00F00F81032A00F01381FB
:1054E000002A40F090815A784D2A00F0C8802FD8C9
:1054F000462A00F0908012D8422A7CD006D8402A52
:105500006DD0412A72D00322A54B66E0442A77D0A1
:10551000452AF8D1D978A34B0520597162E0492A70
:1055200000F096800AD8472A7DD0482AEBD1DB7854
:105530009C49012201F8263F262068E04B2A00F012
:1055400093804C2ADFD1D978964B0220997049E09C
:10555000552A00F0AF8026D8522A00F09A8011D840
:10556000502A00F09180512ACDD18E4D2A7DD2074C
:1055700004D5DB78DB0701D402F0CDFBE178142001
:1055800029752FE0532A00F08C80542ABBD1D3F820
:105590000330012B00F23781E3788249012201F8C0
:1055A0001A3F1A2033E0832A00F097800CD8572A3C
:1055B00000F08C80592AA6D1D3F803307949022211
:1055C00021F8243F242022E0852A00F09080C0F0BA
:1055D0008980FF2A97D1DA78734B1A7038BD40F270
:1055E000FF70D978BDE8384002F02EBCD9786D4BF9
:1055F00000201970F6E7D9786A4B01205970F1E75D
:1056000004221C20D3F80330664941F81C3FBDE852
:10561000384002F078BCD3F803306249042241F8E4
:105620000C3F0C20F3E75F4D042229460820D3F8F5
:10563000033041F8083F02F066FC5C4B1B78002BFE
:10564000CCD12A69A9686879BDE8384003F002B86E
:10565000DA78544B1AB9DA75D97D1720C2E70122DE
:105660004F49DA754A60F7E7D9784E4C0320E1706C
:1056700002F0EAFBE078BDE8384002F0B3BED9782A
:10568000484B15205975ADE7D978464B16209975CA
:10569000A8E7D3F803304349042241F8203F2020F3
:1056A000B5E7404DD3F803302946042241F8103FB6
:1056B0001020C0E7D3F80320012A00F2A480DB7891
:1056C0003849012201F81B3F1B20A0E7DB78354950
:1056D000012201F8273F272099E7D3F80320344B14
:1056E0009A6138BDD3F80320324B1A6038BDD3F825
:1056F00003202F4BDA6138BD5A78D3F803102E4BB4
:1057000043F8221038BD5A78282A64D01CD8022ABF
:105710003AD00CD87AB3012A7FF4F5AED3F803203F
:10572000264B5A6003F0DCF9214B586238BD1C2A25
:1057300046D0272A4AD01B2A7FF4E5AED3F803309F
:105740001E4ADBB2137338BD2B2A4DD008D8292A44
:1057500046D02A2A7FF4D7AED3F80320174BC9E7E7
:105760002D2A4BD045D32E2A7FF4CDAED3F803207B
:10577000124BDA6238BDD3F80320104B1A6003F0E5
:10578000AFF90B4B186238BDD3F803200B4B9A606E
:1057900003F0A6F9064B986238BD00BF280A002026
:1057A0009C0A002008000020960A0020A80E002075
:1057B000B4050020980A0020A80A0020C80E002086
:1057C000D3F80330114ADBB2537338BDD3F803204A
:1057D0000E4B1A6138BDD3F803200C4B5A6138BD0B
:1057E000D3F80320094B7BE7D3F80320074B1A6259
:1057F00038BDD3F80320054B5A6238BDD3F80320D7
:10580000024B9A6238BD04227EE600BFC80E00201B
:105810002DE9FF416423134E134F32783B70D6F8C5
:105820000330212A7A707B6035463C4601F0658260
:1058300000F2C9810E2A00F0928700F24881072AFF
:1058400000F00B8600F22181032A00F019830DD8A5
:10585000012A00F08082022A00F0DC8202232370F9
:10586000AFE200BF280A00209C0A0020052A00F0B1
:10587000008440F22283B2787378002A40F0A48238
:10588000FF2B00F2E285DFE813F0F7030D040F04AD
:1058900017042F0434043A043E04410448044C0421
:1058A00056045E046004620469046D0471047504A6
:1058B00079047D04810483049A049E04A504AC0445
:1058C000B304B704BB04C104C104C804CF04E00599
:1058D000E005E005E005E005E005E005E005E005A0
:1058E000E005E005E005E005E005E005E005E00590
:1058F000E005E005E005E005E005E005E005E00580
:10590000E005E005E005E005E005E005E005E0056F
:10591000E005E005E005E005E005E005E005E0055F
:10592000E005E005E005E005E005E005E005E0054F
:10593000E005E005E005E005E005E005E005E0053F
:10594000E005E005E005E005E005E005E005E0052F
:10595000E005E005E005E005E005E005E005E0051F
:10596000E005E005E005E005E005E005E005E0050F
:10597000E005E005E005E005E005E005E005E005FF
:10598000E005E005E005E005D504E005E005E005FB
:10599000E005E005E005E005E005E005E005E005DF
:1059A000E005D804E005E005E005E005E005E005D8
:1059B000E005E005E005E005E005E005E005E005BF
:1059C000E005E005E005E005E0053B053B053F059A
:1059D000430547054B055705630567056B056F05CF
:1059E000730577057B057F05E005E00583059B05CD
:1059F000E0059D05A405A905E005AB05AF05B305C8
:105A0000B905BD05C105C305CD05D105DE04E10419
:105A1000E504EA04ED04E005E005E005EF04F10427
:105A2000E005D505E005F404F60408050E051205A9
:105A3000E0051605E0051905D90529052B052E05F4
:105A4000DC05E005E005E005E005E005E005E00532
:105A5000E005E005E005E005E005E005E005E0051E
:105A6000E005E005E005E005E005E005E005E0050E
:105A7000E005E005E005E005E005E005E005E005FE
:105A80003105E005E005E00538050A2A00F0EB8461
:105A900008D8082A00F0E484092A7FF4DFAEFFF773
:105AA00015FD8EE10C2A00F01F8640F20586B078C5
:105AB000002840F089817378012B00F03586C0F012
:105AC0002786022B00F0348603233B7079E1182AE5
:105AD00000F090872CD8142A00F0D58616D80F2A0B
:105AE00000F06186132A7FF4B9AE7178B84A0929AB
:105AF00000F29D86DFE811F09806A406A706AA0624
:105B0000AE06B506B806BB06BE06B306162A00F0FA
:105B10006D8740F2D986AF4A516B072900F2518157
:105B2000481C5063106B02EB81018863136348E1EA
:105B30001C2A01F04B8021D81A2A00F0798740F204
:105B40006687A44C94F859206AB9581C4FF00A0093
:105B500004BF9F4B1B685843E06502F0C1FF01235F
:105B6000206684F859306B78042B00F22A81DFE834
:105B700013F07007AC07D707020884071F2A01F04B
:105B8000508001F28C801E2A7FF468AE7078142851
:105B900000F2A285B278002A41F024808E4941F8B3
:105BA00020308E4B9B7E002B00F00B81002800F0F4
:105BB000088100F285108000A0F2146304221944C9
:105BC00002F0A1F9FDE0802A01F0828141D8402A4B
:105BD00001F0548126D8242A01F0ED800CD8222A25
:105BE00001F0E180232A7FF439AE794B1B68C6F8B7
:105BF0000330FFF76BFCE4E0262A01F01981C1F0C5
:105C00000D81272A7FF42AAEB378002B40F0DC8088
:105C10007378142B00F260856D4A11686E4A42F861
:105C20002310CEE0442A01F0478107D8422A01F030
:105C30003F8141F2398103F03FFBC2E0462A01F087
:105C40004381C1F03D81472A7FF408AE03F049FB50
:105C5000B7E0872A01F0D58146D8832A01F0568122
:105C60000AD8812A01F03A81822A7FF4F7AD022214
:105C7000584B83F82C20A4E0852A01F07A81574AFA
:105C800041F2648101255649564C0D709178B3F567
:105C9000006F217081F07381127D12EA050641F0D8
:105CA0006E81184602A901F0F5FF9DF808302672B2
:105CB00063709DF80930A3709DF80A30E3709DF879
:105CC0000E3023719DF80D3063719DF80C30A37177
:105CD0009DF80B30E3712B46E15C227A01330A44D4
:105CE000082B2272F8D16CE08C2A01F0D2811FD8E7
:105CF000892A01F0B381C1F04C818A2A7FF4AEADCC
:105D00007278394B002A41F0C1811A70EB78374A1A
:105D10001370304A92F84811354A11700022354903
:105D20000A7035490A70354A11780B43137048E000
:105D3000F22A01F03382FF2A01F07A828D2A7FF461
:105D40008DAD7278032A01F20F82DFE812F0E209CA
:105D5000C909FB09090AB378002B35D10024284B67
:105D6000284E1C70284B1C7033783BB1274B2621E2
:105D70001A68204603F0BCFFAB78F4540126AC78D7
:105D8000234BD5F803001E55124B002853F824303E
:105D9000B8BF4042984727210246204603F0A8FF9B
:105DA000D5F80330A878002BD8BF02224FF00003AB
:105DB000D6BF01928DE8480000931A46202103F0D7
:105DC00063FF04B0BDE8F08104232370F9E700BF4E
:105DD000880A0020B4050020340A002008000020B2
:105DE0008C0A00208D0A0020B00E0020B80E002082
:105DF000060F0020B30E00203B0F0020B10E002044
:105E0000B20E0020240A0020FC090020200A0020F5
:105E1000F5090020B678002ED6D1A94BA94C1E70EA
:105E2000A94B1E7023783BB1A84B26211A68304637
:105E300003F05EFFAB78E6540126AC78A44BD5F8AE
:105E400003001E55A34B002853F82430B8BF40422E
:105E5000984727210246204603F04AFFD5F8033031
:105E6000A878002BC8BF02224FF00003C6BF0192E2
:105E700000938DE848001A46202103F005FFA0E7B3
:105E8000B578002DA0D1284603F0EEFE0122B078AF
:105E90008F4B27211A542A4603F02AFF0223B07899
:105EA0002A46019300952B46202103F0EDFEB3789E
:105EB000834AD554844AD55483E7B7781FB17278A2
:105EC000022A7FF47EAF00267D4AD6557E4AD655FB
:105ED0006A78012A2ED004D3022A6DD003232370BE
:105EE0006FE77B4CE35D4BB17A4B272103EB8703D4
:105EF0005A68384603F0FCFEAB78E654A878714C3B
:105F0000235C43B1714B262153F8202003F0F0FEAF
:105F10000022AB78E254D5F80320A8782D2103F0B5
:105F2000E7FE0023A8781A4601930093202103F08E
:105F3000ABFE46E7674BDA19127B9846012A35D04B
:105F400003D3022A34D0374604E02D21384603F02B
:105F5000F9FE0746A8785E4E335C43B108EB800338
:105F60005A68272103F0C4FE0022AB78F254A878C7
:105F7000544E335C43B1554B262153F8202003F097
:105F8000B7FE0022AB78F254D5F803602D213E44D1
:105F90003246A87803F0ACFE0023A8781A46019395
:105FA0000093202103F070FE66600AE72121CDE70F
:105FB0003846FEF74FFBCCE7142B3FF705AF3B0607
:105FC00029D5FC077FF5FDAE414C237833B1414B19
:105FD00027215A68304603F08BFE2670394C23780F
:105FE0003BB13A4B26211A68002003F081FE0023C2
:105FF0002370D5F80320384B2D2153F822200020A0
:1060000003F076FE00232021019300931A461846E0
:1060100003F03AFED5E6002F7FF4D6AE2C4C237861
:106020003BB12C4B27215A68384603F061FEAB7810
:10603000E754A878234C235C43B1244B262153F822
:10604000202003F055FE0022AB78E254A878D5F862
:106050000330214A034452F823202D2103F048FE47
:106060000023A8781A4601930093202103F00CFE28
:10607000A7E6FEF7EBFDA4E62D21002003F062FE6B
:106080006060164B1B78002B3FF49BAE144B62688C
:106090001A60144B002A40F0DB811A6842F00802B3
:1060A0001A608EE62121E8E727210A4B1D690020AE
:1060B00003F048FEA847E3E7064B22211D69F6E7F7
:1060C000B20E0020240A0020FC090020200A002033
:1060D000F5090020B4050020340A0020970A0020AA
:1060E000880A0020300A0020AD4B1A695868904792
:1060F000C6E7AB4BAB4A5B6910689847C0E7AA4B51
:106100001B7F6360BDE7A84B5B7FFAE7352100206A
:1061100003F018FEC0F34020B2E70020FEF7C2FBF8
:10612000AEE73521002003F00DFE10F0020F0CBF8A
:1061300001230023E5E73521002003F003FEC043DF
:1061400000F001009CE73421ECE73421F4E734212E
:10615000002003F0F7FDC0F3001091E7904B2421DD
:106160005D69A4E78E4B25211D69A0E78C4B282192
:106170005D699CE78A4B2A215D6998E7884B23215A
:106180001D6994E7864B2B211D6990E72C2174E74C
:106190001521002003F0D6FD002800F02B81834B51
:1061A000B3FBF0F06060AA787F4B03EB42135B7E99
:1061B000002B7FF466AF606804F0FCF960E7784B71
:1061C00033211D6973E73421002003F0BBFDC0F3C8
:1061D000C00055E73421002003F0B4FDC0F3800077
:1061E0004EE73421002003F0ADFDC0F3C02047E7A7
:1061F000002003F04EFF43E7002003F051FF3FE78C
:10620000674B00201D6903F09DF853E71021002023
:1062100003F098FDC0F3034032E76E21002003F045
:1062200091FDC0F309002BE76E21002003F08AFDE9
:10623000000C25E75A4B1B7B63E7002003F01BFF94
:10624000C0F108001CE7584B1B7E5AE7544B564AD6
:106250001B6951E7524B544A1B6950684DE7544B38
:106260001B684EE7534BFBE7382106E74E4B5B8B31
:1062700047E76F21D2E700224F4B7A60197809B1C6
:10628000012179601A704D4B1A781AB1626842F098
:106290000202626000221A70F3E66F21002003F010
:1062A00051FD000EECE60020FEF7D4F9E8E60020F0
:1062B000FEF705FBE4E63C4BDB6822E711210020FA
:1062C00003F040FD08F010F933A3D3E9002308F0F0
:1062D00071F909F015FA08F01DFCD1E63921CCE678
:1062E000314B9B680DE7304B1B690AE700210846DC
:1062F00003F028FD10F0100F19E72B4B5B7E00E731
:10630000002003F005FFBBE6002003F0A6FEB7E681
:10631000002003F0CCFEB3E6002003F0D6FEAFE68B
:10632000002003F0C4FE18B9B07803F0E8FEA7E639
:10633000B07803F0D1FEA3E6002003F0B8FE18B950
:10634000B07803F083FE9BE6B07803F0D1FE97E6C9
:10635000002003F069FE93E6002003F082FF8FE641
:10636000002003F05EFF8BE6002003F061FF87E66C
:10637000002003F04FFF83E6002003F060FF7FE67C
:10638000002003F075FF7BE6002003F05FFF77E657
:10639000002003F077FE73E62D431CEBE236FA3F54
:1063A000B4050020200A0020000A00200024F40088
:1063B000AC0E0020C40E0020FC090020B20E00200C
:1063C0000B215AE66F21002003F0BCFCC0F304400F
:1063D00056E69F4B9F4A1B6950698EE61421D8E60A
:1063E000002003F06BFE4BE6002003F03DFE47E685
:1063F0001321CEE66FF07F436360D4E6002003F004
:10640000C2FF3DE6002003F0C5FF39E6712134E606
:106410000021084603F096FC10F004003FF430AE73
:1064200001236EE6002003F0A7FF29E6002003F019
:106430009CFF25E6002003F08AFF21E6FEF736F8F0
:106440001EE60020FEF758F91AE603233B7018E613
:106450001A6822F008021A60B3E4FEF7E9FBB0E420
:10646000FEF7E6FBADE4B378022B00F0BC80032B13
:1064700000F0BE80002B40F017817378512B00F0A4
:106480008A8027D8472B70D011D8422B63D006D8EA
:10649000402B47D0412B5BD00323237047E0452B93
:1064A0005DD05FD8442BF7D16B4BDB6955E04C2BAB
:1064B00068D007D8492B5FD05AD34B2BECD1664B11
:1064C000DB784AE04F2B60D062D84D2BE4D1624B91
:1064D0005B7D42E0812B6BD014D8552B5ED007D862
:1064E000532B5D4B00F0D08040F2D6809B7E34E091
:1064F000592B56D0802B57D0572BCDD1564B93F8D4
:1065000027302AE0852B60D005D8832B5AD056D966
:10651000524B1B6821E0FE2B02D061D8F02BBBD17F
:106520004F4B16E040F2FF7001F067FD78604D4B75
:106530001B78002B3FF445AC4B4B62681A604B4B09
:10654000002A40F0B3801A6842F008021A6038E46A
:10655000414B1B7801E0404B5B786360E7E73E4BC3
:106560005B79FAE73C4BDB68F7E73B4B9B68F4E76A
:10657000394B93F82630F0E7374BDB7D003318BFFB
:106580000123EAE7344B9B78E7E7334B5B7EE4E794
:10659000314B9B7DE1E7304B1B7DDEE72E4BDB7EF5
:1065A000DBE72D4B9B8CD8E7294B93F82C30D4E7B5
:1065B000274B93F82C30181F43424341CDE7244B1F
:1065C0001B6BCAE7224B9B69C7E743F23901204A9C
:1065D0002748D36900FB0313D36123F00043BCE7D2
:1065E000244B1B78CAE77278234B53F82230B4E768
:1065F0007378282B4AD013D8022B26D006D813B391
:10660000012B7FF449AF1D4B5B68A6E71C2B37D0ED
:10661000272B38D01B2B7FF43FAF184B1B7B9CE7FD
:106620002B2B38D006D8292B33D02A2B7FF434AF2C
:10663000124B3AE72D2B34D030D32E2B7FF42CAFD6
:106640000E4BDB6A89E70D4B63E70C4B8EE700BF0F
:10665000B4050020000A002008000020980A00204D
:10666000FC0E0020970A0020880A0020300A002033
:106670006D4EC641960A0020A80A0020C80E0020D0
:10668000A14B5B7B69E7A04B1B6966E79E4B5B698F
:1066900063E79D4B97E79C4B1B6A5EE79A4B5B6AEF
:1066A0005BE7994B9B6A58E70423F6E61A6822F0E9
:1066B00008021A60FFF785BBB378022B10D17078FF
:1066C000372809D800F5A7709049800004220144BA
:1066D00001F019FCFFF775BB03232370FFF771BBB3
:1066E00004233B70FFF76DBBB378022B0CD170789D
:1066F0003728F1D800F5A7708449800004220144AE
:1067000001F094FCFFF75DBB04233B70FFF759BB1E
:1067100002F012FE20B9B07803F09EFAFFF751BBE9
:1067200006233B70FFF74DBB03F09EFAFFF749BB12
:1067300003F0A2FA764B78601B78002B3FF441AB54
:10674000744B1860744B1A6820B942F008021A6042
:10675000FFF737BB22F008021A60FFF732BBB278AE
:106760002AB1022A08D004233B70FFF72ABB18463F
:10677000FDF77AFEFFF725BB7078072808D81BB90C
:10678000FDF7F6FDFFF71DBBFDF7FAFDFFF719BB9F
:10679000FF28A1D1591C0ABF5E4BD8B21878FDF76B
:1067A000F7FDFFF70EBBB378012B2FD023B1022BDF
:1067B00030D004233B700FE07078082803D8FDF731
:1067C000F8FD606008E00A2816D1544B9B6883F4FA
:1067D0000043C3F3C0337B604D4B1B78002B3FF469
:1067E000F0AA4C4B62681A604B4BBAB91A6842F077
:1067F00008021A60FFF7E5BA0B2802D1FEF714F879
:10680000DFE7FF28E8D1FDF7FDFDDAE7707802F059
:106810000FFAD6E77078FDF7EBFDD2E71A6822F0A1
:1068200008021A60FFF7CDBA1068184410601268A9
:10683000394B12BB1A6842F008021A60FFF7C1BA5E
:106840001068C01AF2E710685843EFE7106890FB31
:10685000F3F0EBE7116891FBF3F003FB1013136007
:10686000E5E710681840E1E710681843DEE71068B4
:106870005840DBE71368DB43F1E71A6822F00802AF
:106880001A60FFF79EBA234A1168234A8B421368A5
:106890000BDA23F0030343F004031360136871B9A8
:1068A00043F008031360FFF78CBA0BBF23F0060315
:1068B00023F0050343F0010343F00203EDE723F067
:1068C00008031360FFF77DBA72780C2A3FF679AAA5
:1068D000DFE802F0071028313A434D565F68717ABD
:1068E00083000D4A126812077FF56BAA0C4A1363E6
:1068F000FFF767BA084A126817073FF562AA084A05
:106900001363FFF75EBA00BFC80E002070050020B9
:10691000970A0020880A0020300A00200010014059
:10692000B4050020AC4A1268D6077FF54AAAAB4AE4
:106930001363FFF746BAA84A1268D5073FF541AA84
:10694000A64A1363FFF73DBAA34A126854077FF5BE
:1069500038AAA24A1363FFF734BA9F4A126812F0AA
:10696000050F3FF42EAA9D4A1363FFF72ABA9A4AED
:10697000126890077FF525AA984A1363FFF721BA9A
:10698000954A126891073FF41CAA944A1363FFF7D3
:1069900018BA914A1268D2067FF513AA8F4A136378
:1069A000FFF70FBA8C4A126897067FF50AAA8B4A3E
:1069B0001363FFF706BA884A126856067FF501AAE4
:1069C000864A1363FFF7FDB9834A126815067FF5FF
:1069D000F8A9824A1363FFF7F4B97F4A1268D40515
:1069E0007FF5EFA97D4A1363FFF7EBB97B4A136389
:1069F000FFF7E7B9794A536B002B3FF4E2A9013B5B
:106A0000536302EB83039B6B1363FFF7DAB973786D
:106A10002E2B04D80121724AD154FFF7D2B9FF2B93
:106A20007FF45AAE01226D4B83F85820FFF7C9B9A5
:106A300073782E2B04D80021694AD154FFF7C1B9CD
:106A4000FF2B7FF449AE0022644B83F85820FFF7F8
:106A5000B8B902F045F8236EC01A0028E36DB8BF3C
:106A6000404298428BBF0023236B84F8593003F1D6
:106A7000FF3398BF2363FFF7A4B9A87803F0FCF8AD
:106A800040B9554A84F85900136823F01003136085
:106A9000FFF797B9E36D9BB102F022F8236EC01A9D
:106AA0000028E36DB8BF4042984209D900234A4A02
:106AB00084F85930136843F010031360FFF781B96D
:106AC000236B013B2363FFF77CB9A878352103F0E2
:106AD00039F910F4007509D000233F4A84F8593081
:106AE000136823F010031360FFF76BB9E36D93B1E4
:106AF00001F0F6FF236EC01A0028E36DB8BF4042D4
:106B0000984208D9344A84F85950136843F0100366
:106B10001360FFF756B9236B013B2363FFF751B9AD
:106B2000A878352103F00EF910F0010509D00023F3
:106B3000294A84F85930136823F010031360FFF7D3
:106B400040B9E36D93B101F0CBFF236EC01A00286A
:106B5000E36DB8BF4042984208D91F4A84F85950A3
:106B6000136843F010031360FFF72BB9236B013B4D
:106B70002363FFF726B9A878352103F0E3F810F076
:106B8000020509D00023144A84F85930136823F011
:106B900010031360FFF715B9E36D93B101F0A0FF87
:106BA000236EC01A0028E36DB8BF4042984208D94E
:106BB000094A84F85950136843F010031360FFF733
:106BC00000B9236B013B2363FFF7FBB80022034BA3
:106BD00083F82C20FFF7F5B8300A0020B405002018
:106BE0000C0F0020FF2A7FF4EFA8A64D70B94FF4D8
:106BF000C364A4F21461204604222944043401F041
:106C000082F9B4F5CD6FF4D1FFF7DBB800F285104F
:106C10008000A0F214610422294401F074F9FFF706
:106C2000D0B8707814283FF657ADB378C3B9954BF8
:106C300053F82020944B7A601B78002B3FF4C1A8B6
:106C4000924B1A60924B2AB91A6842F008021A60F5
:106C5000FFF7B7B81A6822F008021A60FFF7B1B858
:106C6000FF2B7FF4B1A8874D70B94FF4C364A4F231
:106C70001461204604222944043401F0D7F9B4F504
:106C8000CD6FF4D1FFF79DB800F285108000A0F21F
:106C900014610422294401F0C9F9FFF792B8707811
:106CA00014283FF619ADB378190611D5794B9B7EA0
:106CB000002B3FF486A800283FF483A800F285103B
:106CC000754980000422014401F01DF9FFF779B8ED
:106CD000002B7FF479A86F4B9B7E002B3FF471A8AB
:106CE00000283FF46EA800F285106B498000042252
:106CF000014401F008F9FFF764B87278634B0A2A7F
:106D00000CD8DFE802F006151A1F252D32373C415A
:106D1000450062491A6809680A441A601A685C4B9F
:106D2000002A3AD11A6842F008021A60FFF749B8FF
:106D30005A491A680968521AEFE7584A19681268DE
:106D40004A43EAE755491A68096892FBF1F2E4E719
:106D5000524A1868116890FBF1F201FB1202DCE75D
:106D60004E491A6809680A40D7E74C491A68096809
:106D70000A43D2E749491A6809684A40CDE74749BA
:106D80000A68D2430A60C9E71968444A1160C5E736
:106D9000424A196810681860F8E71A6822F0080279
:106DA0001A60FFF70EB8394B1B68C6F80330FDF7C1
:106DB0004DFFFFF706B87378052B3FF602A8DFE812
:106DC00003F0030A11181F26314A136803F00F035A
:106DD0001360FEF7F6BF2E4A136823F0100313600A
:106DE000FEF7EFBF2A4A136823F020031360FEF773
:106DF000E8BF274A136823F040031360FEF7E1BFA2
:106E0000234A136823F080031360FEF7DABF204A99
:106E1000136823F480731360FEF7D3BF71782E29B3
:106E20003FF65AAC1E4A02EB81025366FEF7C9BF19
:106E30001B4B164AD3F820111160D3F82411174ABE
:106E40001160D3F82821D3F82C111A63104A11606D
:106E5000D3F8302193F83C1183F85920D3F834212A
:106E60001A66D3F83821DA650E4A505C08B1012061
:106E70005054002283F84021FEF7A3BF02F019FA14
:106E8000FEF79FBF340A0020970A0020880A0020DE
:106E9000300A00200800002020040020A40A00205E
:106EA000B40500200C0F002002F004FAFEF789BFA1
:106EB00002F001FAFEF785BF02F010FAFEF781BF7B
:106EC00002F00DFAFEF77DBF02F00AFAFEF779BF75
:106ED0000022A74B83F82C20FEF773BF72782AB1EB
:106EE000012A09D003233B70FEF76BBF0122A04BA0
:106EF00083F82C20FEF765BFB3F5006FBEF464AFD6
:106F00009B4981F82C200B63FEF75BBF00234FF0F9
:106F1000FF351946964A974882F8583082F8403132
:106F200002F1640444F82350C15401332F2BF9D1EA
:106F3000914B82F82C101960904B11631960904BA3
:106F4000516382F859101960FEF73BBF127D92071A
:106F50000BD4B3F5006FBEF437AF0421844A82F836
:106F60002C10C2F84431FEF72CBF08233B70FEF70B
:106F700028BF00227E4B83F82C20FEF722BF2B4631
:106F80000022E2540133082BFBD123782372FEF751
:106F900018BF7378012B19D005D3022B1FD0032300
:106FA0003B70FEF70EBF0122764B1A70764B774A84
:106FB0009B781370764B196800230139013311F85F
:106FC000010F082BD054F9D1FEF7FBBE04227B71D0
:106FD000FA712C23EC223B71BA71FEF7F2BE01224A
:106FE000684B6C481A70684B684A9B781370002392
:106FF0000133191811F8091C082BD154F8D1FEF7E8
:10700000E0BE7378032B3EF6DCAEDFE803F002103F
:107010001D22574B93F82C20FA7193F85920D3F87E
:107020004431BA711A0A7A713B71FEF7CABE504BED
:1070300093F82C20FA7193F859201B6BBA711A0A35
:107040007A713B71FEF7BDBE4B4B1B687B60FEF750
:10705000B8BE4A4B1B687B60FEF7B3BE7278002A4D
:107060007EF4AFAEB17800297EF4ABAE40F2D242EE
:1070700093427EF4A6AE40F2FF7000F0E5FE00F011
:107080004AFE0120FDF7CFF9FEF79BBE0122FEF775
:107090003CBE75782DB1012D13D003233B70FEF754
:1070A00090BE042202A940F2FB7000F0BFFF029BD9
:1070B000D6F803209A420ABF01237D607B60FEF769
:1070C00080BEB3782A2B07D10422334940F2FB70EB
:1070D00000F019FFFEF775BE03233B70FEF771BE8B
:1070E0000021234CD4F84C0104F5A87281423EF4EF
:1070F00068AE52F821509D4201F1010520D102EB0A
:107100008503043B0138814214D3C4F84C01FEF7D7
:1071100058BE174AD2F84C1109298FBF0923481CC1
:10712000C2F84C0102EB810294BFC2F850313B70AF
:10713000FEF747BE53F8042F013143F8042CE2E771
:107140002946D3E700231946094AC2F84C3102F513
:10715000A87242F8231001330A2BFAD1FEF731BE90
:107160000A237B60FEF72DBE03233B70FEF729BE8A
:10717000B40500200C0F0020880A0020A40A00207B
:10718000300A00208C0A0020080000208D0A002010
:1071900000000020004000082B0A00207378812B9B
:1071A0007EF40FAEB378922B7EF40BAEB379A32BA3
:1071B0007EF407AE7379B42B7EF403AE3379C52B1E
:1071C0007EF4FFADF378D62B7EF4FBAD1E4B5A68F0
:1071D00042F040525A604FF400425A6102F00CF8FB
:1071E00001F07EFC044601F07BFC001B0028B8BFC8
:1071F0004042B0F57A7FF6DBFDF71CF904F0D4FBD2
:10720000002005F0A1F80021104803F0A0FF0F486E
:1072100003F002FF0E4803F08DFA03F0C9FF4FF0B0
:10722000804005F0EAF80020FDF7FDF8FEF7C9BD43
:1072300040F2D24293427EF4C4AD0122054B83F862
:107240007821FEF7BEBD00BF0010014008000240DB
:1072500000240140B405002000232DE9F041194627
:107260004FF0FF353C4A3D4C13603D4A23631360A9
:107270003C4A636313603C4A84F8593084F85830C0
:1072800084F8403104F1640040F82350D1540133B4
:107290002F2BF9D1354B5B7E002B35D1344B23603E
:1072A0002361A360272100200025636102F04AFDCD
:1072B000304B2621606028461D7002F043FD2E4BA6
:1072C00018602E4B28461D70FDF708FB2846FDF779
:1072D0009BFB2B4B2A461F4643F825200135B5F56D
:1072E000807FF9D1274DAB7EB3B9EB7E23B300236A
:1072F00084F879316B7D6BB3FDF77EFA50B30123CF
:1073000084F82C30BDE8F0811F4B23601F4B2361B4
:107310001F4BA3601F4BC5E74FF4C366DFF87880AF
:10732000A6F21461304604224144043600F07EFE89
:10733000B6F5CD6FF4D1D8E74FF4A766A6F5A761EF
:10734000304604223944043600F070FEB6F5C36FAF
:10735000F4D1CCE70023D3E7880A0020B40500204D
:10736000A40A0020300A00200C0F0020000A002090
:1073700081A60008F5090020200A0020240A002028
:10738000A80A002008000020B5A5000819A60008DA
:10739000F1A5000859A60008340A0020F7B50F4CE3
:1073A00007460E4694E803008DE803000C498A70F6
:1073B0000022C1F803300B4B0F704E701A70FEF7AD
:1073C00027FA21786368084A82F87A119DE8030059
:1073D00084E80300184603B0F0BD00BF9C0A0020FB
:1073E000280A0020970A0020B4050020014B93F8DA
:1073F0007A017047B4050020F7B504461F4A637848
:107400001F4D1370A3780E4695E803005370E37880
:107410008DE80300937023796F46937163795371FC
:10742000A3791371E379D3700022164B1A70FEF71B
:10743000EFF9154B1A782B469AB9327072702A7888
:10744000B2706A78F270EA793271AA7972716A79E7
:10745000B2712A79F27197E8030083E8030003B060
:10746000F0BD012AF7D10948721EF11D10F8014F35
:1074700002F8014F8A42F9D1EDE700BF280A002047
:107480009C0A0020970A00208C0A00208D0A002008
:107490002DE9F047A44B8EB01B78A44C13B994F897
:1074A0007B316BB1A24B1B78063BDBB2192B04D8A6
:1074B000A04A22FA03F3D90702D4002384F8483102
:1074C00094F848319C4E5A1E012A56D8012B14BFFD
:1074D000082307238DF8183094F87C3197498DF8EC
:1074E00019300023CA688DF81A3007923278002AC2
:1074F00038D18B688DF827208DF82030904B197883
:107500008DF8211059788DF82210D9798DF8231033
:1075100099798DF8241059791B798DF825108DF8FB
:107520002630884B1B782BB906A801F017FA0028E3
:1075300000F06F83844BDFF80C821A789946002A9A
:1075400000F03181814B824F1B78013B062B00F20A
:107550002681DFE813F0010101018B0124012401E0
:107560002401B201012ADCD17A48013306AA195C50
:107570001A44082BD171F8D1D3E7032B40D194F8EA
:107580007951002DD6D1337883BBDFF8B0816C4FB1
:1075900098F8020098F801503B7805441D447B7828
:1075A0001D44FB791D44BB791D447B791D443B7907
:1075B0001D4400F0E7FE98F8010000F0E3FE387883
:1075C00000F0E0FE787800F0DDFEF87900F0DAFEF9
:1075D000B87900F0D7FE787900F0D4FE3879EDB2B2
:1075E00000F0D0FE284600F0CDFEA3E7012BA1D18C
:1075F000584F785D013500F0C5FE092DF9D199E7A6
:10760000042B2BD1002301224C4FDFF83481B878B2
:107610007D7888F801300544154488F80020C8F8C2
:10762000043000F0AFFE787800F0ACFE98F800006F
:1076300000F0A8FE98F8010000F0A4FE98F80700FA
:1076400000F0A0FE98F8060000F09CFE98F80500F7
:1076500000F098FEEDB298F80400C1E7072B41D185
:1076600094F87931002B7FF465AF327882BB334BCD
:107670009F7893F80180324B8DF800701D78587810
:107680004744D9798DF802503D449A798DF803002A
:10769000284493F805C08DF80410014493F804E0E1
:1076A0008DF805200A440CEB020373448DF8018029
:1076B0008DF806C08DF807E08DF80830214B1B7857
:1076C000002B3FF437AF0921684601F0C7FD31E7D1
:1076D000012AF3D11F495A5C0DF803200133092B0D
:1076E000F9D1EBE7082B7FF425AF00230120144AE2
:1076F00012495370107053608A7849788DF80020D1
:107700000A4402448DF801108DF802008DF8033010
:107710008DF804308DF805308DF806308DF807307F
:107720008DF80820CAE700BF960A0020B4050020A3
:10773000280A0020110200028C0A00200800002004
:107740009C0A0020A80E00203B0F0020060F0020FE
:10775000B30E00208D0A0020C14A397893688DF855
:1077600036108DF8303080238DF831308A238DF833
:107770003230002307218DF833308DF834308DF806
:1077800035308DF829308DF82A30D3688DF82810DF
:107790000B9398F8003013B90AA801F0DFF8002322
:1077A0003B7089F80030002384F84831337084F846
:1077B0007B3194F8783113B10120FCF734FE94F852
:1077C0007D314BB194F87931B3FA83F35B0984F8D6
:1077D0007931002384F87D3198F80030002B40F097
:1077E000578106A801F006F9002800F051819DF8A4
:1077F0001830062B40F24C819A4B9DF820201A70CD
:107800009DF821205A709DF822209A709DF823201F
:107810009A719DF824205A719DF825201A719DF8BF
:107820002620DA709DF81930079A84F87C318C4B49
:107830001B699A4204BF012384F87B3101F050F99F
:107840000022894B1860894B1A709DF81830072B5D
:107850000CBF0123022384F8483194F82C305A1EBF
:10786000012A50D9052B4ED001224DE0DFF8F0A1BE
:107870003B789AF802009AF8015005440A351D44F5
:1078800000F080FD9AF8010000F07CFD802000F0FF
:1078900079FD8A2000F076FD002000F073FD0020C5
:1078A00000F070FD002000F06DFDEDB2387800F0C2
:1078B00069FD284600F066FD71E780218DF80E1005
:1078C0008A218DF80F100021654A8DF810109378E9
:1078D00050788DF80C303A7803440A3313448DF80D
:1078E000143098F800308DF80D008DF811108DF8D7
:1078F00012108DF81320002B3FF451AF092103A87B
:1079000001F0ACFC4BE70022594B1A7094F82C3074
:10791000042B04D1534B19780A0640F17D8194F869
:107920004821082A04D840F25113D340DF0701D47C
:10793000FDF76EFF94F84831092B6DD101F0D0F8B6
:10794000236A4C4DC01A00282A68B8BF40429042B2
:1079500008D9494B1A78012A04BF02221A7001F093
:10796000BFF8206201F0BCF8636A6A68C01A002898
:10797000B8BF4042904208D93F4B5A78012A04BF11
:1079800002225A7001F0ACF8606201F0A9F8A36A13
:10799000AA68C01A0028B8BF4042904208D9364BA6
:1079A0009A78012A04BF02229A7001F099F8A06225
:1079B00094F8583083B394F840316BBB1D462E4A7F
:1079C0002E48D15C022940F01B8150F823104E1C38
:1079D00000F0158184F83C310023294A1268C4F86C
:1079E0002021284A1268C4F82421226B2163C4F89C
:1079F0002821254A1268C4F82C2194F8592084F8CB
:107A000059300123C4F83021226E84F84031C4F883
:107A10003421E26DC4F8382194F84831092B06D19D
:107A200094F82C20022A04BF052284F82C20D4F8D4
:107A30004C21002A00F0ED80092B40F0EA8094F8F8
:107A40002C30012B40F0E5800023216B0F4850F8CB
:107A500023508D4240F0D980052384F82C30D8E0A3
:107A600008000020280A0020F80E0020A90E00209F
:107A7000970A0020C80E00200C0F002018060020D6
:107A8000880A0020A40A0020300A002004070020F1
:107A900094F87951002D62D103A800F08DFC0028E4
:107AA0005DD000F0A5FC08B184F87E5194F87E21E9
:107AB0009DF80C10531CDBB22244092B84F87E3154
:107AC00082F87F117FF422AF002384F87E31674B68
:107AD00094F87F215978914207D093F82710002914
:107AE0003FF414AF8A427FF411AF93F82730604916
:107AF000934204BF012384F87B3100235A5C013395
:107B00001544082BEDB2F9D194F88731AB4222D15C
:107B1000584B94F880211A7094F881215A7094F887
:107B200082219A7094F883219A7194F884215A7171
:107B300094F885211A7194F88621DA7000F0D0FF4C
:107B40004D4B4E4A186000231370032284F87E3197
:107B500084F8482181E6042384F84831D6E694F875
:107B600079518DBB98F8003073B30AAE304601F0FE
:107B70005FFB48B32B46F25C01331544082BEDB292
:107B8000F9D19DF83020AA42E6D13A4B9DF8292040
:107B90001A709DF82A205A709DF82B209A709DF833
:107BA0002C209A719DF82D205A719DF82E201A7163
:107BB0009DF82F20DA7000F093FF00222E4B186002
:107BC0002E4B1A70072346E694F82C30013B012B0C
:107BD0003FF69CAE236BB3F5006F0CD2FCF70CFEA6
:107BE00048B1206B2349431C236300F053F8092359
:107BF00084F8483138E6002384F82C3086E6D554E2
:107C000001332F2B7FF4DDAE06E701339A427FF478
:107C10001EAF0EB0BDE8F08794F84801082804D8DC
:107C200040F25112C240D207F3D4D4F84401144DAB
:107C3000D3F80330B0F5006F69706B6012D20D4954
:107C400000F038F90B49D4F8440100F0A5F838B138
:107C5000D4F844310133C4F8443165232B70D8E79C
:107C60000723FBE707232B700023F6E6080000201C
:107C700033070020280A0020000F0020050F0020F5
:107C80009C0A0020800000F1006000F5FE300068D2
:107C9000704700000022C0EBC00038B50C4600F56C
:107CA000006503211046FCF759FF0022C5F30721A8
:107CB0001046FCF753FF0022E9B21046FCF74EFFD6
:107CC000002211461046FCF749FF002220701146A1
:107CD0001046FCF743FF0022607011461046FCF787
:107CE0003DFF0022A07011461046FCF737FF00222E
:107CF000E07011461046FCF731FF0022207111465A
:107D00001046FCF72BFF0021607101220846FCF7AA
:107D100025FFA07138BD38B54FF40064012206215B
:107D20000020FCF71BFF002205211046FCF716FF80
:107D3000002101220846FCF711FF8007F3D500223D
:107D400002211046FCF70AFF0022C4F30721104667
:107D5000FCF704FF0022E1B21046FCF7FFFE00250D
:107D6000A5F13F014A424A41002101350846FCF78E
:107D7000F5FE402DF4D1002205211046FCF7EEFE61
:107D8000002101220846FCF7E9FEC307F3D4403482
:107D9000B4F5804FC2D138BDF7B50022C0EBC000AA
:107DA00000F500650C4610460321FCF7D7FE0022C3
:107DB000C5F307211046FCF7D1FE0022E9B21046B8
:107DC000FCF7CCFE002211461046FCF7C7FE00224D
:107DD000074611461046FCF7C1FE00220646114632
:107DE0001046FCF7BBFE0022054611461046FCF784
:107DF000B5FE00228DF8030011461046FCF7AEFEDA
:107E000000228DF8040011461046FCF7A7FE002161
:107E10008DF8050001220846FCF7A0FE23788DF8B6
:107E20000600BB420ED16378B3420BD1A378AB42BC
:107E300008D1DDF80300D4F80330C31A5842584182
:107E400003B0F0BD0020FBE738B5012204460D4623
:107E500000200621FCF782FE002205211046FCF7D7
:107E60007DFE002101220846FCF778FE8207F3D54B
:107E7000002202211046FCF771FE0022C4F3072104
:107E80001046FCF76BFE0022E1B21046FCF766FEDE
:107E9000012229460020FCF761FE00220521104640
:107EA000FCF75CFE002101220846FCF757FEC307E1
:107EB000F3D438BD38B50D46C0EBC00404F50060FE
:107EC0000978FFF7C1FF697804F60100FFF7BCFFEE
:107ED000A97804F60200FFF7B7FFE97804F603007B
:107EE000FFF7B2FF297904F60400FFF7ADFF6979C7
:107EF00004F60500FFF7A8FFA97904F60600BDE81F
:107F00003840FFF7A1BF2DE9F843044688461646DE
:107F1000062101220020FCF721FE00220521104647
:107F2000FCF71CFE002101220846FCF717FE85071E
:107F3000F3D5002202211046FCF710FE0022C4F304
:107F400007211046FCF70AFE0022E1B21046FCF7BA
:107F500005FE0025771EB5420DD1002205211046F1
:107F6000FCF7FCFD002101220846FCF7F7FDC307E2
:107F7000F3D4BDE8F883013414F03F0918F8051074
:107F800039D0781B424242410020FCF7E7FDB9F1AD
:107F9000000F2ED1BD422CD2002205211046FCF745
:107FA000DDFD002101220846FCF7D8FD10F001009C
:107FB000F2D101220621FCF7D1FD00220521104655
:107FC000FCF7CCFD002101220846FCF7C7FD820723
:107FD000F3D5002202211046FCF7C0FD0022C4F3B5
:107FE00007211046FCF7BAFD0022E1B21046FCF76B
:107FF000B5FD0135AFE70122C6E7002210B5032128
:1080000004461046FCF7AAFD0022C4F307211046DF
:10801000FCF7A4FD0022E1B21046FCF79FFDBDE88D
:108020001040002101220846FCF798BDF8B515461E
:10803000002204460E4610460321FCF78FFD002265
:10804000C4F307211046FCF789FD0022E1B2104677
:10805000FCF784FD34467719013DBC4200D1F8BDE0
:108060000021A21BAB1A5A425A410846FCF776FD82
:1080700004F8010BF1E737B5002205211046FCF7A3
:108080006DFD002101220846FCF768FD10F0710427
:10809000F2D100F025FD054600F022FD401B00282E
:1080A000B8BF4042B0F5FA6F18DA74B1264B1B78AE
:1080B000B3B9402225490020FFF7B8FF2022244908
:1080C0004020FFF7B3FF03B030BD40F2FF70FFF771
:1080D00094FFA0F142035C425C41DDE7002CE5D156
:1080E000002140F2FF70FFF7AFFEFFF714FE4022C1
:1080F00016490020FFF707FF202216494020FFF70E
:1081000002FF00234FF4C36402AD45F8043D20464E
:10811000042229460434FFF7F6FEB4F5FF6FF6D1CA
:1081200000234FF4A7640193204604222946043417
:10813000FFF7E9FEB4F5C36FF6D1422140F2FF70BC
:10814000FFF782FEB5E700BFB90E0020080000204F
:10815000000A002060FE000830B5054687B052488E
:1081600004F02AFE01214FF4804003F0C5FE0021F7
:10817000042003F0D9FB03238DF8063018230DEB00
:1081800003048DF807304FF4007324F8143D2146A2
:10819000464803F036FB48238DF807304FF48063E0
:1081A00042482146ADF8043003F02BFB02A804F04E
:1081B00095FE0B2D74D8DFE805F07306585B5E6101
:1081C00064676A6D6F714FF461530293029B02A959
:1081D0005B083548029304F03DFE25230024012569
:1081E0008DF80030072368468DF801308DF8024085
:1081F0008DF8035003F014FC40F2FF312A4804F0DC
:1082000055FF22462821284804F095FE2A4640F2D0
:108210002771254804F08FFE2A4640F22661224845
:1082200004F089FE2A4640F225511F4804F083FEDF
:10823000224640F224411C4804F07DFE224640F6CE
:108240004601194804F077FE224640F66A111648A6
:1082500004F071FE22466021134804F06CFE2946AA
:10826000114804F05CFE07B030BD4FF49643ACE714
:108270004FF4E143A9E74FF41643A6E74FF46143F7
:10828000A3E74FF49633A0E74FF4E1339DE74FF4B3
:1082900061339AE7064B98E7064B96E7064B94E75F
:1082A0004FF4165391E700BF003801400008014029
:1082B00090D0030020A1070040420F00684620F044
:1082C00007018D4619B52A4803889C0604D5294B19
:1082D000DB68190430D58388254803881A0616D52B
:1082E000254B1A689AB9254BDC6A196B8C4239D038
:1082F0004FF400441F490C61196B4C1C1C6319445A
:1083000091F834108180196B202900D11A63184824
:1083100003885B060CD540F2266104F0EBFE174B98
:108320001A6BDB6A9A4202BF4FF40042114B5A614A
:10833000BDE8194085467047104B1A6859680132EC
:10834000202A08BF00228A4205D019688088194473
:10835000C0B208721A600A21094A11609A6A064B73
:108360001A60B9E740F2277104F0E5FDCFE700BFDE
:1083700000380140000801403C0F00203C0700206D
:10838000400F00200A4AD36A116B0133202B08BF2B
:1083900000238B420AD0D16A114481F83400D362A1
:1083A00040F227710122034804F0C5BD704700BFA9
:1083B0003C07002000380140094B59681A68914277
:1083C0000CD05A68511C59601A44127A02705A68CB
:1083D000202A01D100225A600120704700207047F6
:1083E0003C070020014B9862704700BF3C0700200B
:1083F000044B1A7802F0FF0012B1002201201A701B
:10840000704700BF440F002008B5FCF713F80022A6
:10841000034B5A601A60BDE80840FCF709B800BF7A
:108420003C07002010B5441E14F8010F00B910BD20
:10843000FFF7A8FFF8E700BF684620F007018D4668
:1084400031B5254C254B25681B680135082D08BF23
:1084500000259D4286B03AD001A9002002F0C0FC60
:108460009DF80C302268042B1D4B03EB021227D120
:10847000012151702268029903EB021251609DF8AC
:108480000D20022A0CBF01210021226803EB0212F9
:10849000917022689DF80E101201995400222168F3
:1084A00001A8104403EB01111144C07A0132082ADB
:1084B0000872F4D1256006B0BDE8314085467047AA
:1084C000002151702268019903EB0212D6E70020C7
:1084D00002F06CFCEFE700BFD40F0020480F002033
:1084E000540F0020684620F007018D4631B5254C19
:1084F000254B25681B680135082D08BF00259D42C6
:1085000086B03AD001A9012002F06AFC9DF80C3037
:108510002268042B1D4B03EB021227D1012151705D
:108520002268029903EB021251609DF80D20022A85
:108530000CBF01210021226803EB02129170226816
:108540009DF80E10120199540022216801A81044D0
:1085500003EB01111144C07A0132082A0872F4D1E8
:10856000256006B0BDE83140854670470021517056
:108570002268019903EB0212D6E7012002F016FCF3
:10858000EFE700BFD40F0020480F0020540F002059
:10859000684620F007018D462B4B11B52B4A196810
:1085A000126887B0914208D10021012002F04AFBF5
:1085B00007B0BDE81140854670471968244A02EBB0
:1085C0000111497801F0FF00002930D004218DF815
:1085D0000C1000210191196802EB01114968029108
:1085E000196802EB0111897801F0FF0041B3022103
:1085F0008DF80D1019680901515C8DF80E100021DD
:10860000186802EB00100844047A01A808440131FC
:108610000829C472F4D11A6801A801321A601A68D4
:10862000082A04BF00221A6002F018FBC0E719688C
:108630008DF80C0002EB0111496802900191CFE71F
:108640008DF80D00D6E700BF500F00204C0F002022
:10865000D80F0020F0B501388BB00E4615460C231C
:10866000072800F20E81DFE810F00A010801060178
:10867000040102010C010001080002228DF81430EF
:1086800003238DF815300023ADF816208DF8133034
:1086900002F0ECF901214FF0007003F039FC0121E8
:1086A000084603F029FC0121082003F025FC0021E5
:1086B000082003F039FC01214FF4EA1003F034F9EB
:1086C00003238DF8063018238DF807304FF400731C
:1086D0000AAC24F8243D2146814803F092F8042393
:1086E0008DF807304FF480730127214600247C4821
:1086F000ADF8043003F085F803A88DF812408DF82A
:108700000C408DF80D708DF80E408DF80F408DF8EF
:1087100010708DF8117002F0B6F9B6F5006F8DF893
:1087200018408DF819408DF81A7080F2AC807301F2
:10873000ADF81C304FF6FF73ADF81E40ADF8203099
:10874000ADF82230ADF824408DF8267006A802F06E
:10875000F7F9012300228DF818308DF819208DF8D3
:108760001A30002D00F09E80B5F5006F80F29A80DF
:10877000ADF81E204FF6FF726901ADF81C10ADF880
:108780002020ADF82220ADF824308DF8263006A840
:1087900002F0D6F902238DF818307313F60046F074
:1087A000040600270124ADF81E604FF6FF7606A8E8
:1087B000ADF81C308DF819708DF81A40ADF82060B6
:1087C000ADF82260ADF824708DF8264002F0B8F9BB
:1087D0000323BD428DF818308DF819708DF81A40BA
:1087E0006FDD6B13ED0045F00405ADF81C30ADF8FE
:1087F0001E50ADF82060ADF82260ADF824408DF831
:10880000264006A802F09CF901240726002514231F
:1088100002A88DF808308DF809608DF80A508DF89F
:108820000B4003F0FDF8152302A88DF808308DF8F1
:1088300009608DF80A508DF80B4003F0F1F813230E
:1088400002A88DF808308DF809608DF80A508DF86F
:108850000B4003F0E5F82146022002F0F3F921462F
:10886000102002F0EFF90BB0F0BD042206E7102251
:1088700004E7142202E7282200E76422FEE6C82269
:10888000FCE60822FAE64FF6FF73ADF81C40ADF89F
:108890001E40ADF82030ADF82230ADF824408DF800
:1088A000264053E74FF6FF71ADF81C20ADF81E20AF
:1088B000ADF82010ADF82210ADF824308DF8262048
:1088C00065E70423ADF81C70ADF81E30ADF82060EC
:1088D000ADF82260ADF824408DF8267091E700BF16
:1088E000000C014037B50021022002F0ABF9002155
:1088F000102002F0A7F90021012002F0A3F90024C2
:108900000725142301A88DF804308DF805508DF843
:1089100006408DF8074003F083F8152301A88DF871
:1089200004308DF805508DF806408DF8074003F0AF
:1089300077F8132301A88DF804308DF805508DF8D1
:1089400006408DF8074003F06BF802F08FF82146DF
:108950004FF0007003F0DCFA03B030BDF0B543789F
:1089600087B004464268002B37D004238DF80C30C2
:10897000002302920193A37803B102238DF80D30F6
:10898000234613F8081B06AA02F80A1D04F1100179
:1089900013F8010B8B4202F8010FF9D101A802F084
:1089A0005DF9042816D1104F104B3D681B68013546
:1089B000082D08BF00259D4214D03B680C4E06EBE5
:1089C000031694E80F0086E80F00012108463D6079
:1089D00002F038F9012007B0F0BD8DF80C3001929B
:1089E0000293C8E70020F6E74C0F0020500F00204C
:1089F000D80F002030B50C4B0C4C054622681B6884
:108A00009A420FD02268531C2360094B03EB0213D8
:108A10000FCB85E80F002368082B01D100232360CA
:108A2000012030BD002030BDD40F0020480F0020B1
:108A3000540F0020684620F007018D4601B5BDE8BF
:108A400001408546704700BF684620F007018D460B
:108A500001B5124B19781A46E9B15B681049013328
:108A600053600B6801330B600E4B196811B1196824
:108A700001391960002313700B4B1A683AB11A6858
:108A8000013A1A601B6813B90122084B1A70BDE83D
:108A900001408546704701221A70EDE790070020DB
:108AA000980A00203C0F0020400F0020440F0020B7
:108AB00008B5042003F022FC48F6A04003F02AFC8D
:108AC000012003F02DFC05480022032103F07CF86F
:108AD000BDE80840012003F037BC00BF9AC3020084
:108AE000014B5868704700BF90070020000000004D
:108AF0002DE9F041002403254FF0090892B001A9A7
:108B000045488DF80740ADF804808DF8065002F016
:108B100078FE01A941488DF80740ADF804508DF862
:108B2000065002F06EFE0121084603F0D9F901213A
:108B30004FF4007003F0E0F9394802F06DFA394B58
:108B400004270793384B07A9089380230C934FF40D
:108B500080730D934FF480630E9320230F934FF493
:108B600000532F48109309940B9411940A9702F024
:108B7000C3FA01212A4802F0EAFA01264FF46023E1
:108B800002A92A480294049305948DF80C608DF88C
:108B90000D608DF8187001F0FBFD2B46324629461A
:108BA000224801F06DFE2B46022241461F4801F08B
:108BB00067FE2B462A4608211C4801F061FE2B4621
:108BC00021463A46194801F05BFE22464FF4FC610B
:108BD000164801F01CFE3146144801F00FFE3146E4
:108BE000124801F002FE114801F01AFE0F4C204617
:108BF00001F01BFE0028FAD10C4801F01AFE0B4CC4
:108C0000204601F01BFE0028FAD10121074801F09F
:108C100019FE12B0BDE8F08100080140000C0140CF
:108C2000080002404C240140980700200024014025
:108C3000F8B50A2863D8DFE800F006626262626273
:108C400062620A125F003C4B188880B2F8BD3A4B52
:108C5000588883B240F26E2058430013F8BD364B5B
:108C6000D88880B206F084F805F050FC0022334B1F
:108C700005F0A0FC24A3D3E9002305F09BFC0446E7
:108C80000D4602460B4620A1D1E9000105F0DEFAAF
:108C90001FA3D3E9002306460F462046294605F0C8
:108CA000B3FD02460B463046394605F0ADFD05F0F2
:108CB00059FF05F02BFC0022214B05F0A5FD06F025
:108CC0003BFE15A3D3E9002305F074FC14A3D3E9FC
:108CD000002305F0BDFA02460B4613A1D1E90001BD
:108CE00005F092FD12A3D3E9002305F0AFFA05F0D9
:108CF00039FF06F0E5F9F8BD0F4B9888A9E7002089
:108D0000F8BD00BFAFF300806666666666660A401F
:108D10009A99999999990140C3F5285C8FA272405C
:108D20000000000000FEAA409A999999FD6F2F411A
:108D3000C3F5285C8F127140980700200000303F77
:108D4000000024400022014B1A607047A007002059
:108D5000034B9B7A13B10522024B5A60704700BF48
:108D600064100020A00700200422014B5A607047C5
:108D7000A0070020034B1A7A202A04BF00221A728F
:108D8000704700BFA00700207047212810B508D108
:108D9000114B1B681B7803F07F03212B19D0022095
:108DA00010BD2028FBD10C4B0C4A1B681B7810729D
:108DB00003F07F03212B0A4B18BF0023002BEED0BA
:108DC0000024054A20461268936154829847204641
:108DD00010BD044BF4E700BFC4100020A007002022
:108DE0001D8E0008358E0008074B1B681B7803F0AA
:108DF0007F03212B06D100F0DF00022814BF0220E0
:108E00000020704702207047C410002021B90128BB
:108E10008CBF0220002070470220704720B9082232
:108E2000024B1B681A82704701487047C41000202B
:108E300048000020FFF7F2BF08B5032005F0B2F9A3
:108E4000064B0246D8604FF48871054804F0A2FE34
:108E5000BDE80840032004F06BBF00BFA00700205E
:108E6000CA10002038B50024C025324B20461B68AC
:108E70009C725D72DC7204F0C9FE4FF400712046F2
:108E800004F0E1FE1021204604F0F4FE40212046CB
:108E900005F094F88021204605F07EF8204604F085
:108EA00077FF254B204693F8341005F028F820462C
:108EB00004F03EFF2146012004F0C5FE29460120B2
:108EC00005F06AF82021012004F0D4FE214601209B
:108ED00004F0E5FE4FF4C061022004F0B4FE4FF44C
:108EE0008071022005F058F82146022004F0D7FED8
:108EF0002021022004F0BEFE2146032004F0A3FE40
:108F00004FF48871032005F059F84021032004F044
:108F1000F6FF4FF44051032004F0C1FE2146032028
:108F200004F0A8FE204604F0C7FC0122034B5A605F
:108F300038BD00BFC410002048000020A00700205A
:108F4000014904F0C5BA00BF80000020014904F0C7
:108F5000BFBA00BF88000020054B1B68DB78042BDC
:108F600004D8044901EBC30104F0B2BA00207047F1
:108F7000C41000209000002008B5002002F03AFF45
:108F8000BDE8084001214FF4000002F0C1BF0322F8
:108F9000014B5A60704700BFA0070020044B9A7A2B
:108FA000044B12B105225A6070470122FBE700BF53
:108FB00064100020A0070020202110B1024802F018
:108FC0008CBC014802F08BBC000C01407047684625
:108FD00020F007018D4679B5134C144E2368144DCB
:108FE0009BB23380288831880140480505D54FF66B
:108FF000FF3323600F4BDB68984733882A88134080
:10900000990507D54FF6FF530B4923600B7C0133BD
:10901000DBB20B7433881A40130401D504F0B2FCA0
:10902000BDE8794085467047445C00405A100020F6
:109030000A11002048000020A007002008B52021C8
:10904000074802F04AFC01220020064B06491A603C
:10905000064A186010604FF4E0520A801A6008BD9A
:10906000000C0140405C00400A110020445C0040BC
:1090700010B50024074B1B689C72FFF7DFFF064BFF
:10908000064A1C604FF406431380054A1360054BE3
:109090005C6010BDC4100020445C00400A11002038
:1090A000405C0040A007002038B501230024054D96
:1090B00020462B60044B1C60FFF77EFF03232046F5
:1090C0002B6038BD405C0040445C0040074A136898
:1090D0009BB243F00803136013689BB243F0040390
:1090E00013600322024B5A60704700BF405C00408F
:1090F000A007002008B54FF6FB7305490A68134026
:109100000B60FFF74BFF4FF406430B6008BD00BF39
:10911000405C004010B51D4C072818BF2070237814
:10912000052B06D8DFE803F003070B101823FFF721
:10913000E1FF062306E0FFF7DDFF042302E0022340
:1091400063700323237006E06378013BDBB2637036
:109150006378002BF1D010BD0D4A13689BB243F029
:1091600010031360052323700A23637010BD637816
:10917000013BDBB263706378002BECD14FF6EF73E9
:10918000034A11680B401360D3E700BFC8100020EA
:10919000405C0040142307B58DF8043000238DF89F
:1091A00005308DF80630012301A88DF8073002F054
:1091B00037FC03B05DF804FB07B5FFF7DDFEFFF7F2
:1091C000E9FF04F0C5FB0121082002F095FE2023F1
:1091D000ADF8043003238DF80630102301A90448AC
:1091E0008DF8073002F00DFB03B05DF804FB00BF03
:1091F000000C0140FFF7CEBFFFF756BF0A4B30B55A
:109200000446D86878B15A68052A0BD10022074D68
:10921000D9688A4202D30022DA6030BD515DA15480
:109220000132F5E7002030BDA0070020CA10002061
:10923000084A10B5D368082B0AD90023064C195DDB
:10924000C1540133092BFAD100230120D36010BD92
:10925000002010BDA0070020CA10002010B5074C48
:109260008AB22160C02104F083FC2188012004F02F
:1092700025FEBDE81040012004F04BBDA0070020F2
:10928000704710B5FFF72CFC074C2368C01AB0F5E7
:10929000FA7F07D9054AD36883F40063D360FFF7E8
:1092A0001FFC206010BD00BF0C110020000C01400D
:1092B0007047704770477047054B064AD3F8031054
:1092C000054B19B99B889BB2536070471B89FAE71D
:1092D000280A00209C0A0020006C0040704770475C
:1092E000704710B5FBF7E2F805280E4C0ED80123A5
:1092F00063600D4B1B7843B10C4B62681A600C4BDA
:1093000062B91A6842F008021A6010BDFBF7CEF885
:1093100040F2F9339842EAD80023E9E71A6822F0CC
:109320000802F1E79C0A0020970A0020880A002022
:10933000300A002000000000014B1878704700BF81
:10934000B4070020024B03EB80004068704700BF69
:10935000B40700202DE9F74F754CE36993B1754DC3
:109360002E787EB9FFF7BCFB734B1B68C01A002830
:10937000E369B8BF4042984204D9304601F0FAF898
:1093800001232B70236A93B16C4D2E787EB9FFF7C1
:10939000A7FB6B4B1B68C01A0028236AB8BF40426A
:1093A000984204D9304601F0E5F801232B70FFF70D
:1093B00097FB644C237B04EB83039B68C01A002853
:1093C000B8BF40420A2823DDFFF78AFB2121074668
:1093D000207B00F0B7FC0646257B04EB8505286959
:1093E000301A05F0C9FC8046A868381A05F0C4FC9C
:1093F0000146404605F0C8FD05F088F84AA3D3E9C8
:10940000002305F0D7F805F085FBAF6068602E619A
:109410003521207B00F096FC10F0400705460DD06A
:10942000207B01F0A7F80121237B474AD154474A0A
:109430000F33D15C012904BF0221D154207B444E5B
:1094400006EB40135B69002B59D0222100F07AFC17
:1094500094F80C80002806EB48135B69B8BF4042C3
:1094600098424CD904EB08031B7D6BB9342140466C
:1094700000F068FC342140F48062404600F038FC83
:109480000122237B23441A75637DDFF8CCB06BB9CE
:1094900098465FFA88F0FAF78CFF0BF8080008F19D
:1094A0000108B8F1080FF4D1012363754FF02708C4
:1094B0004FF0000902222749DFF890A05FFA89F0F7
:1094C0008DE80600FAF775FF9DE806001BF80930E5
:1094D00083424AD009F1040351F823300BF8090004
:1094E000022B3BD0032B03D0012B3ED100283CD0D4
:1094F0001AF80830012B08BF0AF8082035E094F864
:109500000C8004EB08031B7D002BBDD034214046AA
:1095100000F018FC342120F48062404600F0E8FBA3
:10952000237B00222344AEE7FCA9F1D24D62904098
:1095300008000020050F0020000F0020A90E0020C9
:10954000F80E0020B4070020FC0900200C0F0020BA
:10955000000A0020C80E0020CA07002028B91AF807
:109560000800012801D10AF8083009F10109B9F110
:10957000080F08F10108A1D1237B15F0010104EBCC
:10958000030200F0D580917F71B901219177774A6C
:109590001A44127BD20707D58B40754A1B33D15C26
:1095A000012904BF0221D154237B15F0020104EBF1
:1095B000030200F0CA80D17F81B90121D1776B4AC3
:1095C0001A44527B12F0010F08D0694A0E3312F888
:1095D0001310012904BF022102F8131015F08001B5
:1095E00000F0C080237B624A0333D05C012801D1A4
:1095F0000220D05447B1237B5D4A0F33D05C012851
:1096000001D10220D054F9B1DFF870E1207B9EF83F
:10961000003043FA00F2D10711D50121DFF860C113
:1096200001FA00F28CF80020DFF858C18CF8001025
:109630005049097819B923EA02038EF800308022D4
:10964000352100F055FB27B140223521207B00F069
:109650004FFB207B06EB40131B690BB36A051FD43D
:10966000392100F06FFB21210746207B00F06AFBC7
:10967000237B381A06EB431200281269B8BF404218
:1096800090420DD9184600F075FF0121237B3A4A1C
:10969000D154374A1533D15C012904BF0221D1547A
:1096A000207B06EB4013DB6803B36B051ED4FAF78F
:1096B000D1FF21210546207B00F044FB237B281AA3
:1096C00006EB43160028F268B8BF404290420DD91D
:1096D000184600F04FFF0121237B274AD154244A2A
:1096E0001533D15C012904BF0221D154FFF7F8F9E9
:1096F000236AC01A0028B8BF40420A2804DDFAF7DE
:1097000009FFFFF7EDF92062FBF776F840BB2578FB
:1097100035B900F0A9FA284600F02CFF0123237088
:10972000207B00F05FF80023237303B0BDE8F08FC7
:10973000907F00283FF438AF91770C4A1A44127B8F
:1097400090077FF531AF5B0027E7D07F00283FF41B
:1097500045AFD177054A1A44527B12F0020F33E726
:109760000023DCE7002F3FF474AF44E7C80E00206D
:109770000C0F0020B00E0020B20E0020B80E00200A
:10978000B30E00203B0F002073B5134E0446335C2C
:109790000D463BB1114B262153F8202000F0A8FACA
:1097A0000023335585EAE572A2EBE57220462721B6
:1097B00000F09EFA01220A4B002D1A554FF00003CB
:1097C000D8BF02220093019220211A46204600F0C1
:1097D0005BFA02B070BD00BF240A0020200A0020FE
:1097E000F50900202DE9F04F352185B0044600F041
:1097F000A9FA0346C04861014618327ED6F80480B3
:1098000012F0400F18BF41584FEA530B03F0010507
:1098100017BF0BF0010950F801A05FFA85FBC1F1F9
:10982000000A12BFC8F100085FFA85F90BF0010BBE
:10983000150602F03F060393204613D5FBF732F8D6
:10984000B0FA80F77F09721E039B072A00F27B8122
:10985000DFE812F00E000E000E000E0012011201E1
:1098600012011201FBF71EF8071C18BF0127EAE7D7
:10987000A24D2A5D013A0E2A00F26581DFE812F05E
:109880000F001E002D003B004B00540063007200CF
:10989000A200C400CA006301F800E101DC01342128
:1098A000204600F04FFA012205EB84035860023E87
:1098B000934B96421A551BD802231AE005EB8403FA
:1098C0005A6842F002023421204600F011FA514653
:1098D0002046FFF759FF03230BE0BBF1000F00F018
:1098E00032812121204600F02DFA864B43F82400D6
:1098F00004232B5527E105EB84035A6842F001024B
:109900003421204600F0F4F9CAF100012046FFF7A7
:109910003BFF0523EDE7B9F1000F00F0148120466D
:1099200000F028FE0623E4E705EB84035A6834219F
:10993000204622F0030200F0DBF941462046FFF703
:1099400023FF0723D5E7B9F1000F40F0FC8049461B
:109950002046FFF719FFC8F100012046FFF714FF6A
:109960000823C6E7B9F1000F00F0ED802121204661
:1099700000F0E8F9064600212046FFF705FF614A9E
:10998000342152F8243020469B1B42F8243005EB4A
:1099900084035A6822F0030200F0AAF94246272104
:1099A000204600F0A5F932462D21204600F0A0F90E
:1099B00000232021019300931A46204600F064F909
:1099C000092396E7990540F1BE802121204600F049
:1099D000B9F94D4B002118602046FFF7D5FE002253
:1099E0002D21204600F084F900222121204600F09C
:1099F0007FF9033E00223921204600F079F9012E3B
:109A000038D8C8F10001B2E0B9F1000F00F09B8036
:109A10000B236EE7B9F1000F40F09580212120461D
:109A200000F090F9494606462046FFF7ADFE05EBEB
:109A300084035A68342122F00302204600F058F9CA
:109A400042462721204600F053F902222D2196FBA1
:109A5000F2F2204600F04CF94B46CDF80490CDF8D8
:109A600000901A462021204600F00EF90D2340E711
:109A70009A0568D50E233CE7204D2A5D013A0E2A4F
:109A800061D8DFE802F008192A4354606360608BF4
:109A90009579B9DED9000122194B342120461A5597
:109AA00000F050F905EB8403062E58603FF404AF34
:109AB000082E7FF41DAFFFE6062E05D105EB8403CB
:109AC0005A6822F00302FCE6082E7FF400AF05EB93
:109AD00084035A6822F00302F5E6731F012B07D8AE
:109AE000BBF1000F04D0062E3FF402AF0F2300E7B6
:109AF0004FB30C23FDE600BF000A0020D80700206A
:109B0000F5090020AC0E0020C40E0020052E05D162
:109B100005EB84035A6822F00302EFE6072E7FF478
:109B2000F3AE05EB84035A6822F00302E8E6731FE4
:109B3000012B05D8B9F1000F02D0052ED6D1BBE616
:109B4000002F7FF4FEAE05B0BDE8F08F002FFAD1F4
:109B5000073E012E0AD905EB84035A68342122F00E
:109B6000030242F00202204600F0C2F841462046BD
:109B7000FFF70AFE0A23BCE6002FE4D1073E012EC0
:109B80007FF63FAF05EB84035A68342122F00302CD
:109B900042F00102204600F0ABF832E7002FD2D0AD
:109BA0002121204600F0CEF805EB840398602FE7D2
:109BB000002FC8D12121204600F0C4F8064605EB4D
:109BC0008409D9F80420342122F00302204600F051
:109BD0008FF842462721204600F08AF8D9F808205D
:109BE0002D2116440222204696FBF2F200F080F866
:109BF000019700973B4634E79B05A4D50E2321210E
:109C000020462B5500F09EF8124B0021186020468C
:109C1000FFF7BAFD204600222D2100F069F820460A
:109C20000022212100F064F800223921204605B0ED
:109C3000BDE8F04F00F05CB800212046FFF7A4FD1E
:109C400018E705EB84035A683421204600F050F8E9
:109C500000234EE6C40E0020024B1A5C0AB9012212
:109C60001A547047D8070020024B1A5C0AB10F2221
:109C70001A547047D8070020014B185C704700BF8A
:109C8000D8070020000000002DE9F84391461F4648
:109C900080460E46002241F0800101209DF82050B0
:109CA0009DF82440FAF75AFF002249460120FAF7AE
:109CB00055FF394600220120FAF750FF29460022BD
:109CC0000120FAF74BFF01222146104647EA0927F7
:109CD000FAF744FF45EA072506F07F06034B4644A2
:109CE00044EA052443F82640BDE8F883E407002051
:109CF00070B5144606460D46002241F08001012051
:109D0000FAF72CFF0022210E0120FAF727FF00228C
:109D1000C4F307410120FAF721FF0022C4F3072111
:109D20000120FAF71BFF0122E1B21046FAF716FFF5
:109D300005F07F05024B354443F8254070BD00BF58
:109D4000E407002038B5264B01F07F055B5D002B52
:109D500041D0002229460120FAF700FF002201200D
:109D60001146FAF7FBFE002201201146FAF7F6FE33
:109D7000002201201146FAF7F1FE012200211046CF
:109D8000FAF7ECFE002201201146FAF7E7FE002266
:109D900001201146FAF7E2FE0022040211460120DA
:109DA000FAF7DCFE0022044311460120FAF7D6FE42
:109DB00001222402044300211046FAF7CFFE2402B8
:109DC000222D40EA040001D0422D08D1030206D51D
:109DD00040F07F4038BD034B054453F8250038BDA3
:109DE00031FF0008E407002070B50B4C054622182F
:109DF00092F800220E465AB96C21FFF7A3FF06F035
:109E00000F0320F00F021A436C212846FFF770FF62
:109E1000631983F8016270BDE407002038B50C4671
:109E20006C210546FFF78EFF240104F0700420F03A
:109E3000700222432846BDE838406C21FFF758BF26
:109E400038B50C466C210546FFF77CFFE40304F4AB
:109E5000C03420F4C03222432846BDE838406C218B
:109E6000FFF746BF38B50C466C210546FFF76AFF81
:109E7000240504F4700420F4700222432846BDE84F
:109E800038406C21FFF734BF38B50C466C210546CD
:109E9000FFF758FF240604F0706420F0706222433C
:109EA0002846BDE838406C21FFF722BF38B50D4683
:109EB0006C210446FFF746FF3DB140F0804220464A
:109EC000BDE838406C21FFF713BF20F08042F6E771
:109ED00038B50D466C210446FFF734FF3DB140F420
:109EE00000222046BDE838406C21FFF701BF20F476
:109EF0000022F6E738B50D466C210446FFF722FF35
:109F00003DB140F480222046BDE838406C21FFF787
:109F1000EFBE20F48022F6E738B50D466C210446EA
:109F2000FFF710FF3DB140F480422046BDE83840C5
:109F30006C21FFF7DDBE20F48042F6E738B50D4610
:109F40006C210446FFF7FEFE3DB140F4005220466E
:109F5000BDE838406C21FFF7CBBE20F40052F6E795
:109F600038B50D466C210446FFF7ECFE3DB140F4D8
:109F700080522046BDE838406C21FFF7B9BE20F47E
:109F80008052F6E738B50C466C210546FFF7DAFE3D
:109F9000230748BF20F070004FEA04124CBF40F482
:109FA000006020F4076002F0700202436C21284632
:109FB000BDE83840FFF79CBE38B50C466C2105461D
:109FC000FFF7C0FEE40104F4F06420F4F0622243E1
:109FD0002846BDE838406C21FFF78ABEFFF7ECBF8A
:109FE00038B50D466C210446FFF7ACFE3DB140F09C
:109FF00000522046BDE838406C21FFF779BE20F0C2
:10A000000052F6E738B50D466C210446FFF79AFE7C
:10A010003DB140F080522046BDE838406C21FFF74A
:10A0200067BE20F08052F6E708B5074B034493F86B
:10A0300000222AB96C21FFF785FE00F00F0008BD51
:10A0400093F8010208BD00BFE407002008B56C21A9
:10A05000FFF778FEC0F3021008BD08B56C21FFF7CA
:10A0600071FEC0F3C13008BD08B56C21FFF76AFE70
:10A07000C0F3035008BD08B56C21FFF763FEC0F3C1
:10A08000036008BD08B56C21FFF75CFEC0F380706B
:10A0900008BD08B56C21FFF755FEC0F3C04008BDF0
:10A0A00008B56C21FFF74EFEC0F3804008BD08B52F
:10A0B0006C21FFF747FEC0F3803008BD08B56C2166
:10A0C000FFF740FEC0F3403008BD08B56C21FFF734
:10A0D00039FEC0F3003008BD08B56C21FFF732FE31
:10A0E000C0F30213020548BF43F00803184608BD39
:10A0F00008B56C21FFF726FEC0F3C31008BDFFF7BB
:10A10000F7BF08B56C21FFF71DFEC0F3407008BD16
:10A1100008B56C21FFF716FEC0F3007008BD38B516
:10A120000C466D210546FFF70DFE640104F0600446
:10A1300020F0600222432846BDE838406D21FFF739
:10A14000D7BD38B50C466D210546FFF7FBFD64030E
:10A1500004F4C04420F4C04222432846BDE83840FD
:10A160006D21FFF7C5BD38B50C466D210546FFF7DB
:10A17000E9FD240204F4706420F47062224328464E
:10A18000BDE838406D21FFF7B3BD38B50C466D21F1
:10A190000546FFF7D7FD04F00F0420F00F0222431D
:10A1A0002846BDE838406D21FFF7A2BD38B50D4601
:10A1B0006D210446FFF7C6FD20F47F0040EA05420A
:10A1C0006D212046BDE83840FFF792BD38B50D46F9
:10A1D0006D210446FFF7B6FD3DB140F40042204634
:10A1E000BDE838406D21FFF783BD20F40042F6E75B
:10A1F00038B50D466D210446FFF7A4FD3DB140F092
:10A2000080722046BDE838406D21FFF771BD20F017
:10A210008072F6E708B56D21FFF794FDC0F3411099
:10A2200008BD08B56D21FFF78DFDC0F3413008BDB5
:10A2300008B56D21FFF786FDC0F3032008BD08B502
:10A240006D21FFF77FFD00F00F0008BD08B56D21FF
:10A25000FFF778FD0314D8B21B0648BF60F0FF007B
:10A2600008BD08B56D21FFF76DFDC0F3C03008BD16
:10A2700008B56D21FFF766FDC0F3006008BD38B575
:10A280000C4670210546FFF75DFD04F0030420F441
:10A29000401242EA04522846BDE838407021FFF7D8
:10A2A00027BD38B50D4670210446FFF74BFD3DB183
:10A2B00040F400222046BDE838407021FFF718BD69
:10A2C00020F40022F6E738B50D4670210446FFF76A
:10A2D00039FD3DB140F480222046BDE83840702170
:10A2E000FFF706BD20F48022F6E738B50C46702152
:10A2F0000546FFF727FD04F0030420F4403242EA4C
:10A3000004422846BDE838407021FFF7F1BC38B55B
:10A310000D4670210446FFF715FD20F47F4040EA0A
:10A32000052270212046BDE83840FFF7E1BC38B572
:10A330000D4670210446FFF705FD20F0FF0045EAB9
:10A34000000270212046BDE83840FFF7D1BC08B5B7
:10A350007021FFF7F7FCC0F3015008BD08B570216C
:10A36000FFF7F0FCC0F3C04008BD08B57021FFF74F
:10A37000E9FCC0F3804008BD08B57021FFF7E2FC9E
:10A38000C0F3014008BD08B57021FFF7DBFCC0F346
:10A39000072008BD08B57021FFF7D4FCC0B208BD86
:10A3A00070B50E466F2115461C46FFF7CBFC16B163
:10A3B000C0F30903336015B1C0F304432B700CB133
:10A3C000000E207070BD37B5FEF78AFB0446FEF71D
:10A3D00087FB001B0028B8BF40420928F7DD002199
:10A3E00013220846FFF784FC022253238DE80C0059
:10A3F0000022412310466C21FFF746FC062503236B
:10A400008DE82800002309211A461846FFF73CFC76
:10A4100000240A2101230191224620460094FFF7DF
:10A4200033FC3F4A1021537F2046DB080193137F02
:10A430002246DB0800930723FFF726FC394A7021E8
:10A440002046FFF755FC2046FFF7EEFD364B83F81C
:10A450000102042083F80042FDF714FC01301CD0F7
:10A460000520FDF70FFC0B2102462046FFF740FCBC
:10A470002846FDF707FCC1B22046FFF7B5FC0720D0
:10A48000FDF700FCC1B22046FFF7C8FC0820FDF72D
:10A49000F9FBC1B22046FFF78FFD002220211046B4
:10A4A000FFF726FC00222D211046FFF721FC002299
:10A4B00021211046FFF71CFC012223210020FFF779
:10A4C00017FCDC2224210020FFF712FC46F6DB02F9
:10A4D00025210020FFF70CFC40F2B71226210020B6
:10A4E000FFF706FC4DF2B71227210020FFF700FC12
:10A4F00040F2B71228210020FFF7FAFBDC222A21C4
:10A500000020FFF7F5FB0A222B210020FFF7F0FBCC
:10A5100014210020054A03B0BDE83040FFF7E8BB36
:10A52000000A00201E000CC4E4070020FFFF0F00FB
:10A5300038B5074C044494F8001241B994F801521C
:10A54000FFF752FC012384F8015284F8003238BD31
:10A55000E4070020064B034493F8002232B10022A6
:10A5600093F8011283F80022FFF73EBC704700BF4A
:10A57000E407002037B501250C4BC4B21D540C4B29
:10A5800000221D5427212046FFF7B2FB20464FF63C
:10A59000FF722621FFF7ACFB0023019500931A46BA
:10A5A00020212046FFF770FB03B030BDF5090020E5
:10A5B000240A0020002808B50BDB03F095FF0AA34E
:10A5C000D3E9002304F020F905F02AF904F0A2FAF7
:10A5D00008BD03F089FF04A3D3E9002304F014F9B4
:10A5E00005F08EF8F2E700BF34F7FFFF7F84EE3FFF
:10A5F00008B503F079FF06A3D3E9002304F004F9BA
:10A6000005F00EF904F086FA08BD00BFAFF3008034
:10A61000EB1100A2941A5D40002808B50BDB03F093
:10A6200063FF0BA3D3E9002303F0C4FF05F068F830
:10A6300004F070FA08BD03F057FF05A3D3E9002327
:10A6400003F0B8FF05F0ECF8F2E700BFAFF30080CD
:10A6500034F7FFFF7F84EE3F08B504F08DFB03F075
:10A6600055FF05A3D3E9002303F0A4FF05F048F844
:10A6700004F050FA08BD00BFEB1100A2941A5D402F
:10A68000704700BF7047FEE7FEE7FEE7FEE7704752
:10A690007047704770477047704770477047704702
:10A6A00070477047704770477047704770477047F2
:10A6B00070477047704770477047014B1B681847D9
:10A6C000B40E0020014B1B68184700BF080F002084
:10A6D000014B1B68184700BFBC0E0020014B1B68D4
:10A6E000184700BFC00E0020704770477047704782
:10A6F00070477047704770477047704770477047A2
:10A700007047704770477047704770477047704791
:10A710007047704770477047704770477047704781
:10A720007047704770477047704770477047704771
:10A73000704700BF08B5154B984213D003F5A053DE
:10A74000984218D0A3F5C05398421DD101214FF46F
:10A75000007001F0E9FB00214FF40070BDE80840F3
:10A7600001F0E2BB01214FF4806001F0DDFB00212C
:10A770004FF48060F2E701214FF4004001F0D4FB78
:10A7800000214FF40040E9E708BD00BF0028014068
:10A7900043680A7923F4702323F4807343EA022385
:10A7A0000A6810B5134343608A68CB688468134312
:10A7B000084A224013434A7943EA420383600A7CF1
:10A7C000C36A013A23F47003D2B243EA0253C3626C
:10A7D00010BD00BFFDF7F1FF00230360037143715B
:10A7E0008360C360012303747047836819B143F029
:10A7F00001038360704723F00103FAE7836819B10E
:10A8000043F480738360704723F48073FAE7C9B21E
:10A81000436812B119434160704723EA0101FAE726
:10A82000836843F00803836070478068C0F3C0000A
:10A830007047836843F00403836070478068C0F307
:10A8400080007047836819B143F4A00383607047A8
:10A8500023F4A003FAE78068C0F380507047436890
:10A86000013923F4604343EA41334360704743684E
:10A8700019B143F400634360704723F40063FAE7BF
:10A88000092970B51BD90726A1F10A04C56804EB94
:10A890004404A64025EA060503FA04F42C43C460E8
:10A8A000062A18D81F24013A436B02EB8202944017
:10A8B00023EA040301FA02F21A43426370BD07243B
:10A8C000056901EB4106B44025EA040503FA06F4E4
:10A8D0002C430461E4E70C2A0CD81F24073A036BCD
:10A8E00002EB8202944023EA040301FA02F21A43C3
:10A8F000026370BD1F240D3AC36A02EB82029440CA
:10A9000023EA040391401943C16270BD836819B101
:10A9100043F480138360704723F48013FAE7C06C1C
:10A9200080B27047014B1868704700BF4C2401404B
:10A93000436819B143F480634360704723F4806334
:10A94000FAE7436819B143F480534360704723F436
:10A950008053FAE7836823F4E0431943816070472A
:10A96000836819B143F400438360704723F40043C4
:10A97000FAE7836819B143F402138360704723F444
:10A980000213FAE78068C0F340507047092970B598
:10A990001CD90726A1F10A04C56804EB4404A640AB
:10A9A00025EA060503FA04F42C43C460836B0232E3
:10A9B000C3F30154121B1F24D2B202EB8202944053
:10A9C00023EA040391401943816370BD072405699C
:10A9D00001EB4106B44025EA040503FA06F42C43D2
:10A9E0000461E3E7836B013923F4401343EA015325
:10A9F00083637047425070472830405880B2704798
:10AA0000436823F4400323F4007319434160704703
:10AA1000416282627047436823F01F03194341601B
:10AA20007047054B9A6818B142F400029A6070476B
:10AA300022F40002FAE700BF002401400368194233
:10AA400014BF012000207047C9430160704743686C
:10AA5000006810EA112004D0C9B2194214BF0120C5
:10AA6000002070476FEA11210160704708B501218D
:10AA70004FF0007001F064FABDE8084000214FF08B
:10AA8000007001F05DBA01232C4A1360536813F083
:10AA9000010351D00378012B13680CBF43F08003EE
:10AAA00023F0800313604378012B244B1A680CBFFA
:10AAB00042F0400222F040021A608278012A1A68AD
:10AAC0000CBF42F0200222F020021A60C378012B52
:10AAD0001A4B1A680CBF42F0100222F010021A60E2
:10AAE0000279012A1A680CBF42F0080222F008021B
:10AAF0001A604379012B114B1A680CBF42F0040213
:10AB000022F004021A60C37982791B0643EA827339
:10AB1000027A43EA0243427A43EA02534289013A03
:10AB20001343064AD361136823F00103136050688E
:10AB3000C04300F0010070471846704700640040B1
:10AB400030B501250378364A9D40ADB2EC43D2F8CA
:10AB5000001241F00101C2F80012D2F81C1221408B
:10AB6000C2F81C128178002934D1D2F80C12DB0013
:10AB70002140C2F80C124289C18841EA024103F126
:10AB8000804202F5C842C2F840128388018943EA34
:10AB90000143C2F8443243782149A3BBD1F80432BF
:10ABA0002340C1F8043283891D4A83BBD1F8143293
:10ABB0001C40C1F81442837B012B02BFD2F81C3227
:10ABC0002B43C2F81C32D2F8003223F00103C2F842
:10ABD000003230BD0129DED1D2F80C12DB0029434E
:10ABE000C2F80C128188C28803F1804342EA014214
:10ABF00003F5C843C3F840220189428942EA014271
:10AC0000C3F84422C7E7D1F804322B43C9E7012B2C
:10AC100002BFD2F814322B43C2F81432CBE700BF84
:10AC2000006400400023037043708370C37003719D
:10AC300043718371C371032303720223437201239F
:10AC400043817047044B5A6911B1104358617047F2
:10AC500022EA0000FAE700BF006400402A4B0246E7
:10AC60009968F0B5480132D49968090148D49B68C5
:10AC7000DB0047D40420F0BD1168D3F8806149059A
:10AC8000116021433143C3F88011917A01F00F0123
:10AC90009172D3F8844124F00F04C3F88441D3F8AF
:10ACA00084412143C3F88411D2F80B4005F180415F
:10ACB00001F5C841C1F88841D2F80F20C1F88C21B4
:10ACC000D3F8802142F00102C3F88021F0BD0020BA
:10ACD000050105F1804303F5C843D3F8801101F065
:10ACE0000101C3F88011117A547A0029C4D0566842
:10ACF000D3F88071F6003143214356603943C2E7EF
:10AD00000120E5E70220E3E700640040012814D0B9
:10AD100003D302281FD000230CE016498B688A68F1
:10AD200089689B0003F00403C1F380610B4302F0C8
:10AD300002021343104AD05C70470E498B688A6840
:10AD40009B09120A02F0020203F0040313438A680B
:10AD5000C2F3C062EDE707498B688A689B0B120C4F
:10AD600002F0020203F0040313438A68C2F3007284
:10AD7000DFE700BF00640040B1FF0008012809D0F0
:10AD800002D302280BD07047074A936843F0800330
:10AD900093607047044A936843F40043F8E7024A1B
:10ADA000936843F40003F3E700640040034B202260
:10ADB00008B9DA6070471A61704700BF006400404C
:10ADC00020B9064BD86800F003007047012802D173
:10ADD000024B1869F7E70020704700BF006400408D
:10ADE000030103F1804202F5C84210B4D2F8B04129
:10ADF00004F004040C72B4BBD2F8B041640D0C60D2
:10AE0000D2F8B04103F1804304F002044C72D2F84E
:10AE1000B44103F5C84304F00F048C72D2F8B42196
:10AE200010BC120ACA74D3F8B821CA72D3F8B82178
:10AE3000120A0A73D3F8B821120C4A73D3F8B82156
:10AE4000120E8A73D3F8BC21CA73D3F8BC21120A3C
:10AE50000A74D3F8BC21120C4A74D3F8BC311B0E0F
:10AE60008B74FFF7A3BFD2F8B041E4084C60C7E78A
:10AE7000044B1A6842F002021A601868C0F34000DE
:10AE8000704700BF00640040054B1A6822F00202C0
:10AE90001A60186880F00200C0F34000704700BFDD
:10AEA00000640040034B9B69034214BF0120002053
:10AEB000704700BF00640040024A936923EA000023
:10AEC0009061704700640040202840D011D80628C7
:10AED0002ED005D8042835D0052824D0002070476E
:10AEE00007282AD00828F9D1214BD868C0F30010D0
:10AEF0007047B0F5007F30D007D840282AD0B0F591
:10AF0000807FEBD11A4B98690FE0B0F5803F2CD0D1
:10AF1000B0F5003F26D0B0F5806FDFD1144B9869B3
:10AF2000C0F380007047124B986800F00100704732
:10AF30000F4B9868C0F3002070470D4B9868C0F322
:10AF4000004070470A4BD868C0F3C0007047084BF8
:10AF50001869F9E7064B1869C8E7054B9869C0F30B
:10AF600040007047024B5868C0E7014B5868EBE758
:10AF700000640040202835D00CD8062826D004D8FC
:10AF8000042829D005281DD07047072821D008287B
:10AF900026D07047B0F5007F30D005D8402825D0A6
:10AFA000B0F5807F24D07047B0F5803F2BD0B0F54E
:10AFB000003F2CD0B0F5806F28D1164A936923F05A
:10AFC000040319E00122134B9A6070474FF480721A
:10AFD000F9E74FF48032F6E708220E4BDA6070474B
:10AFE0001022FAE708220B4B1A6170471022FAE789
:10AFF000084A936923F0010393617047054A9369F6
:10B0000023F00203F8E70822024B5A60704710222F
:10B01000FAE700BF00640040036823F00103036007
:10B020000023036043608360C3602D4B984243D08C
:10B0300011D83C3B984230D006D8283B984222D0C9
:10B040001433984224D07047264B98422AD01433A8
:10B0500098422CD07047244B98423AD008D8A3F598
:10B06000677398422ED003F5627398422FD07047D1
:10B070001E4B98422FD0143398422ED0283B984232
:10B080001FD11B4A0AE01B4A536843F00F0317E025
:10B09000184A536843F0F00312E0164A536843F429
:10B0A00070630DE0134A536843F4704308E0114A9B
:10B0B000536843F4702303E00E4A536843F470036B
:10B0C000536070470B4A536843F07063F8E7084ACF
:10B0D000DAE7074ADDE7064AE5E7054AE8E700BFA1
:10B0E0006C000240440002401C0402404404024040
:10B0F00000040240000002408B6810B50C6A026830
:10B1000023430C6922F4FF4223434C6922F070026E
:10B1100023438C692343CC6923434C6A23438C6AC1
:10B12000234313430360CB6843600B6883604B6821
:10B13000C36010BD0023036043608360C36003618C
:10B1400043618361C3610362436283627047036842
:10B1500019B143F001030360704723F00103FAE7DC
:10B16000036812B119430160704723EA0101FAE74D
:10B17000406880B27047C3004CBF044B044B1B684F
:10B18000034214BF01200020704700BF00040240AA
:10B1900000000240FFF7EFBFC3004CBF014B024B62
:10B1A000586070470004024000000240FFF7F4BFFF
:10B1B0000022044B1A605A609A60DA60024A5A61AF
:10B1C000704700BF00040140FFFF0700827930B5DF
:10B1D0000168037942B3CC43184A03F180431568F0
:10B1E00003F582332540156055682C4054601C6877
:10B1F0002143196003689468D9430C409460D46873
:10B200002140D1604179102906D19168194391609C
:10B21000D1680B43D36030BD01F1804202F5823228
:10B2200011680B43136030BD03F1804303F5823393
:10B230001A6822EA0101196030BD00BF0004014014
:10B2400000230C2203600371427183717047024A2C
:10B25000136918431061704700040140034B5B6998
:10B26000034214BF01200020704700BF00040140CA
:10B27000014B5861704700BF00040140054B1A683C
:10B280005B69034004D0024214BF012000207047D4
:10B290001846704700040140014B5861704700BFD9
:10B2A00000040140044B1A6802F038021A601A6860
:10B2B00010431860704700BF00200240044B1A681A
:10B2C00022F008021A601A6810431860704700BF25
:10B2D00000200240044B1A6822F010021A601A681B
:10B2E00010431860704700BF00200240034B044A1F
:10B2F0005A6002F188325A60704700BF0020024055
:10B3000023016745024A136943F0800313617047C4
:10B3100000200240014BD86980087047002002409D
:10B32000014B186A704700BF00200240024BD869E9
:10B33000C0F34000704700BF00200240024B186875
:10B34000C0F34010704700BF00200240044B1A6950
:10B3500011B110431861704722EA0000FAE700BFFC
:10B36000002002400128064B03D1D86900F00100FB
:10B370007047DB68184214BF01200020704700BFEF
:10B3800000200240014BD860704700BF00200240FF
:10B39000084BDA68D10709D4DA68520708D4DB68A9
:10B3A00013F0100F14BF03200420704701207047D2
:10B3B000022070470020024073B504460025FFF7C5
:10B3C000E7FFFF2601280FD114B9052002B070BD98
:10B3D00001950196019B1BB9FFF7DAFF013CF1E7EC
:10B3E000019B013B0193F5E7002C08BF0520EDE729
:10B3F00038B5054640F6FF70FFF7DEFF042815D18B
:10B400000B4C40F6FF70236943F002032361656132
:10B41000236943F040032361FFF7CEFF012805D0E5
:10B42000236923F00203DB04DB0C236138BD00BF7A
:10B430000020024010B540F6FF70FFF7BDFF042862
:10B4400014D10B4C40F6FF70236943F004032361D1
:10B45000236943F040032361FFF7AEFF012805D0C5
:10B46000236923F00403DB04DB0C236110BD00BF60
:10B470000020024010B540F6FF70FFF79DFF042842
:10B480002BD1164C164B40F6FF70A36003F18833A6
:10B49000A360236943F020032361236943F0400341
:10B4A0002361FFF789FF04280FD1A52223690F200C
:10B4B00023F02003DB04DB0C2361236943F010033A
:10B4C0002361084B1A80FFF777FF012805D0236915
:10B4D00023F01003DB04DB0C236110BD00200240CD
:10B4E0002301674500F8FF1F70B506460F200D4683
:10B4F000FFF762FF042818D10C4C0F20236943F09A
:10B5000001032361ABB23380FFF756FF042804D157
:10B510002D0C75800F20FFF74FFF012805D0236900
:10B5200023F00103DB04DB0C236170BD002002402B
:10B5300070B505460F200E46FFF73EFF042810D1D8
:10B54000084C0F20236943F0010323612E80FFF78D
:10B5500033FF012805D0236923F00103DB04DB0C52
:10B56000236170BD0020024070B506460F200D46D5
:10B57000FFF722FF042816D10B4C0C4BADB2A36091
:10B5800003F18833A36023690F2043F01003236184
:10B590003580FFF711FF012805D0236923F0100340
:10B5A000DB04DB0C236170BD0020024023016745F2
:10B5B00010B504460F20FFF7FFFE04282AD1E4430C
:10B5C000204B214AE1B29A6002F188329A601A69EE
:10B5D000FF2942F010021A6113D1C4F30723FF2B95
:10B5E00019D1C4F30743FF2B1DD1240EFF2C22D108
:10B5F0000420144A136923F01003DB04DB0C1361ED
:10B6000008E0124B0F201981FFF7D6FE0428E4D082
:10B610000128EED110BD0D4A0F205381FFF7CCFE5B
:10B620000428DED0F4E7094A0F209381FFF7C4FE17
:10B630000428DAD0ECE7054BA4B2DC810F20FFF739
:10B64000BBFEE5E7002002402301674500F8FF1F2D
:10B6500038B5054640F6FF70FFF7AEFE042839D135
:10B660001D4C1E4B40F6FF70A36003F18833A360AE
:10B67000236943F020032361236943F040032361DE
:10B68000FFF79AFE04281DD1236923F02003DB0471
:10B69000DB0C2361236943F010032361104B7DB160
:10B6A00000221A8040F6FF70FFF786FE012811D0B5
:10B6B000094A136923F01003DB04DB0C136138BD66
:10B6C000A522EEE7012805D0236923F02003DB043F
:10B6D000DB0C236138BD00BF002002402301674519
:10B6E00000F8FF1FF8B5124C124B0546A36003F19A
:10B6F0008833A3600F200E461746FFF75DFE04282F
:10B7000014D1236947F0F80743F0100323613E4347
:10B71000094B35435D800F20FFF74EFE012805D011
:10B72000236923F01003DB04DB0C2361F8BD00BFA9
:10B73000002002402301674500F8FF1F08B5294B90
:10B74000984236D015D8A3F50063984223D003F56C
:10B750008063984226D0A3F50063984240D101212E
:10B76000042000F0E1FB00210420BDE8084000F0C7
:10B77000DBBB1D4B984223D003F58063984226D053
:10B78000A3F5006398422BD10121402000F0CCFBAF
:10B7900000214020E9E70121082000F0C5FB00213D
:10B7A0000820E2E70121102000F0BEFB002110205C
:10B7B000DBE70121202000F0B7FB00212020D4E7A7
:10B7C0000121802000F0B0FB00218020CDE7012185
:10B7D0004FF4807000F0A8FB00214FF48070C4E7A4
:10B7E00008BD00BF00140140001C0140012108B544
:10B7F000084600F099FBBDE808400021012000F058
:10B8000093BBCB782DE9F041DA0648BF8A780E88E1
:10B8100003F00F0548BF154316F0FF0F1AD00021A3
:10B820004FF0010E4FF00F0C02680EFA01F737EAE5
:10B8300006040BD18C000CFA04F822EA080205FA7F
:10B8400004F4282B42EA040225D14761013108297A
:10B85000EBD10260FF2E1CD900214FF0010E4FF0FA
:10B860000F0C426801F108040EFA04F434EA0607EA
:10B870000BD18F000CFA07F822EA080205FA07F745
:10B88000282B42EA07020AD1446101310829E9D193
:10B890004260BDE8F081482B08BF0761D6E7482B1E
:10B8A00008BF0461F1E74FF6FF7303800223837042
:10B8B0000423C37070478368194214BF012000201D
:10B8C0007047806880B27047C368194214BF012076
:10B8D00000207047C06880B27047016170474161C5
:10B8E00070470AB10161704741617047C16070479C
:10B8F00041F4803383618161836183698369704727
:10B90000054A136823F07F031B041B0C194341EA0B
:10B9100000111160704700BF00000140014B18602A
:10B92000704700BF1C00204230B5134A00F4401598
:10B93000B5F5401F536884B20ED1556823F070638B
:10B9400025F07065556021B1400D000104FA00F04A
:10B950000343094A536030BDC2024DBF0322420D6A
:10B960001201C0F303454CBFAA4004FA02F223EAD5
:10B97000020343F07063E6E70000014010B50F24B6
:10B9800001F0030301F0FC0101F1804101F5803178
:10B990008A689B009C4022EA04028A608A68984078
:10B9A0001043886010BD00BF6FF070424FF0FF3150
:10B9B000094BC3F88010C3F88420C3F88011C3F882
:10B9C00084210022104602F1C00101320F2A43F8FF
:10B9D0002100F8D1704700BF00E100E04FF0206285
:10B9E000084B09495A6000229A60D9601A615A616D
:10B9F0009A61DA611A625A624FF0FF329A62DA6231
:10BA00001A63704700ED00E00000FA0540F0BF60E7
:10BA1000024B40F40030D860704700BF00ED00E0FA
:10BA200030B5C37802786BB31C4BD9684378C943EF
:10BA3000C1F30221C1F10404A3400F2424FA01F14F
:10BA4000FF24807801400B4302F0FC0101F16041CA
:10BA500001F5614102F00300D1F80053C0001B0161
:10BA600083406B4004FA00F003406B40C1F80033A0
:10BA70000123510902F01F0203FA02F2084B43F8B6
:10BA8000212030BD0121530902F01F0201FA02F208
:10BA90000349203341F8232030BD00BF00ED00E012
:10BAA00000E100E00023037043708370C3707047AF
:10BAB000F8F753BBF8F753BBF8F753BBF8F753BB92
:10BAC0000001F8F752BBF8F753BB024B5868C0F3BC
:10BAD0000930704700ED00E0012300F01F029340A1
:10BAE0004009044A403052F8202093430CBF012003
:10BAF0000020704700E100E0014B1860704700BF74
:10BB000000EF00E00122430900F01F0002FA00F0FC
:10BB1000024A603342F82300704700BF00E100E0B2
:10BB2000024B5868C0F30900704700BF00ED00E009
:10BB3000012300F01F0293404009044A803052F86C
:10BB4000202093430CBF01200020704700E100E05B
:10BB5000014B1868704700BF00ED00E021F0604124
:10BB600021F07F01014B01439960704700ED00E037
:10BB7000014A024BDA6070470400FA0500ED00E06C
:10BB8000014A024BDA6070470100FA0500ED00E05F
:10BB9000044B1A6911B110431861704722EA000082
:10BBA000FAE700BF00ED00E0012300F01F0003FAF8
:10BBB00000F0044B5A6A11B110435862704722EAF0
:10BBC0000000FAE700ED00E0114B30B5DC68FF251E
:10BBD000E443C4F30224C4F1040325FA04F49940B5
:10BBE00004EA02030B43C0F30121C0F3811080007B
:10BBF00000F1604000F56D408269C9008D4022EA85
:10BC00000505856182691B018B401343836130BD4B
:10BC100000ED00E00123C0F3832003FA00F0044BA1
:10BC20005B6A30EA03030CBF01200020704700BFAD
:10BC300000ED00E000F01F010120034B88405A682E
:10BC400010435860704700BF00ED00E000F01F0097
:10BC5000431E0120024A98405168084350607047D3
:10BC600000ED00E00123C0F3833003FA00F0044B41
:10BC70005B6A30EA03030CBF01200020704700BF5D
:10BC800000ED00E0C0F38143094A0BB9D06A704768
:10BC9000012B0AD1C0F30153906ADA00D040022B85
:10BCA00014BF00F00F00C0B27047106B704700BFA8
:10BCB00000ED00E0034B10F4800F0CBF586B986B45
:10BCC000704700BF00ED00E00C4B1A6842F0010223
:10BCD0001A6059680A4A0A405A601A6822F0847247
:10BCE00022F480321A601A6822F480221A605A689C
:10BCF00022F4FE025A6000229A607047001002404F
:10BD00000000FFF80C4BB0F5803F1A6822F4803237
:10BD10001A601A6822F480221A6003D0B0F5802FCE
:10BD200005D070471A6842F480321A6070471A686A
:10BD300042F4A022F9E700BF00100240034A136852
:10BD400023F0F80343EAC00010607047001002407F
:10BD5000014B1860704700BF00004242034A53681D
:10BD600023F47C13194301435160704700100240D3
:10BD7000014B1860704700BF60004242034A53689D
:10BD800023F0030318435060704700BF00100240C7
:10BD9000024B586800F00C00704700BF00100240D2
:10BDA000034A536823F0F00318435060704700BF04
:10BDB00000100240034A536823F4E06318435060C4
:10BDC000704700BF00100240034A536823F46053D9
:10BDD00043EAC0005060704700100240044B1A78DC
:10BDE00011B110431870704722EA0000FAE700BF53
:10BDF00009100240014B1860704700BFD800424252
:10BE0000034A536823F4404318435060704700BF0F
:10BE1000001002400022064B01281A701A7002D04E
:10BE2000042802D070471870704705221A707047B6
:10BE300020100240014B1860704700BF800442424E
:10BE4000024A136A18431062704700BF0010024094
:10BE5000014B1860704700BF3C0442421C4A10B5B9
:10BE6000536803F00C03042B01D0082B1FD0194B8F
:10BE7000036053681849C3F30313CC5C0368E340C1
:10BE800043605468C4F302240C5D23FA04F4846014
:10BE90005468C4F3C2240C5DE340C3605268C2F32B
:10BEA000813211440A7CB3FBF2F3036110BD536885
:10BEB0005168C3F38343CC0303F1020302D407495F
:10BEC0004B43D5E751688903F9D40249F8E700BF2D
:10BED0000010024000127A00B9FF000800093D007E
:10BEE000044B5A6911B110435861704722EA0000AF
:10BEF000FAE700BF00100240044B9A6911B11043E9
:10BF00009861704722EA0000FAE700BF0010024083
:10BF1000044BDA6911B11043D861704722EA00007E
:10BF2000FAE700BF00100240044BDA6811B1104379
:10BF3000D860704722EA0000FAE700BF0010024014
:10BF4000044B1A6911B110431861704722EA0000CE
:10BF5000FAE700BF00100240014B1860704700BFB5
:10BF600040044242014B1860704700BF4C004242FF
:10BF7000014B1870704700BF071002404209012AA8
:10BF8000074B07D11B6800F01F0023FA00F000F0F8
:10BF900001007047022A0CBF1B6A5B6AF3E700BF0F
:10BFA0000010024010B540F2FF140A493120FFF79B
:10BFB000E5FF08704B6801334B600B7813B94B6891
:10BFC000A342F3D13120FFF7D9FF003018BF012081
:10BFD00010BD00BFE8090020024A536A43F0807395
:10BFE0005362704700100240034B9B68184214BF15
:10BFF00001200020704700BF00100240014B187064
:10C00000704700BF0A10024008B5164B98421FD077
:10C0100003F5744398420FD0A3F57843984220D19A
:10C0200001214FF48040FFF78BFF00214FF4804047
:10C03000BDE80840FFF784BF01214FF48050FFF7AF
:10C0400073FFBDE8084000214FF48050FFF76CBF3C
:10C0500001214FF40040FFF773FF00214FF400402F
:10C06000E6E708BD003C0040038810B503F44152E8
:10C070004C880B8823438C882343CC8823430C892A
:10C0800023434C8923438C892343CC892343134383
:10C090009BB20380838B23F400631B041B0C8383FC
:10C0A0000B8A038210BD838BF0B523F47B6323F0EE
:10C0B0000F031B041B0C8383022303840B89868BD1
:10C0C000022B87B005460C46B6B23AD08B8801A841
:10C0D000002B14BF02270127FFF7C0FEE388228947
:10C0E000B3F5007F4FF00A0301991CBF7F017A432B
:10C0F00003FB01F308BF1202B3FBF2F30A2205337C
:10C100009BB2B3FBF2F303F001021202C3F34F033D
:10C11000991E89B2FE2924BF002202231343E2881C
:10C1200013439BB262882B8423881343A28843F471
:10C1300000631343628913431E43B6B2AE8307B054
:10C14000F0BD0022E4E70023038043808380C380A6
:10C15000038143818381C3810723038270470023C6
:10C160000222038043808380C38002814381704721
:10C17000038821B19BB243F040030380704723F052
:10C1800040031B041B0CF8E7838B21B19BB243F4E3
:10C1900080638383704723F480631B041B0CF8E7E0
:10C1A0000B0901219940838889B29BB212B11943CE
:10C1B0008180704723EA0101FAE783889BB212B1BC
:10C1C00019438180704723EA0101FAE781817047B2
:10C1D000808980B270474FF6FF63994203880BBF96
:10C1E00023F480739BB21B0443F4807308BF1B0CC1
:10C1F00003807047838821B19BB243F0040383809E
:10C20000704723F004031B041B0CF8E7038823F496
:10C2100000631B041B0C038003889BB2194301803D
:10C22000704703889BB243F48053038070470388B0
:10C2300021B19BB243F400530380704723F40053B1
:10C240001B041B0CF8E7012914BF008B808A80B205
:10C250007047008A80B270470388B1F5804F15BFE0
:10C2600023F480439BB21B0443F4804318BF1B0C90
:10C27000038070470389194214BF012000207047D2
:10C28000202906D1038903889BB243F04003038031
:10C290007047402901D0082901D103897047C9435B
:10C2A00089B201817047012310B58488008901F0AB
:10C2B0000F0280B203FA02F21040A4B205D00909BD
:10C2C0008B401C4214BF0120002010BD552906D10F
:10C2D000038903889BB243F04003038070475629CB
:10C2E00001D0532901D103897047012301F00F01C7
:10C2F0008B40DB439BB20381704700BF044B042893
:10C300001A680CBF42F0040222F004021A6070475F
:10C3100010E000E0014B5860704700BF10E000E003
:10C320000128084B04D11A6842F001021A607047D4
:10C33000023003D11A6822F00102F7E700229A6066
:10C34000704700BF10E000E0044B1A6818B142F0DB
:10C3500002021A60704722F00202FAE710E000E0E1
:10C36000014B9868704700BF10E000E0C308022B43
:10C37000044B0CBF1B68DB6823FA00F000F00100DF
:10C38000704700BF10E000E030B5048C42EA0313B0
:10C3900024F001042404240C0484048B058C24F070
:10C3A000F3042404240C1C4325F002031B041B0C7F
:10C3B00041F00101A4B20B430483038430BD30B5C6
:10C3C000048C120224F010042404240C0484058B31
:10C3D000048C42EA033324F0200225F44075120451
:10C3E0002D05120C2D0D42EA01111D4341F01001E3
:10C3F000ADB289B20583018430BD08B5314B984296
:10C4000040D014D8A3F5006398422DD003F5806383
:10C41000984230D0B0F1804F52D101210846FFF749
:10C420008FFD00210120BDE80840FFF789BD264BA4
:10C43000984235D004D8A3F58063984229D008BD2E
:10C44000224B984204D003F5006398422FD008BDD8
:10C4500001214FF40060FFF767FD00214FF40060F9
:10C46000BDE80840FFF760BD01210220FFF768FD2D
:10C4700000210220D7E701210420FFF761FD002100
:10C480000420D0E701210820FFF75AFD00210820F1
:10C49000C9E701211020FFF753FD00211020C2E75A
:10C4A00001212020FFF74CFD00212020BBE70121C6
:10C4B0004FF40050FFF738FD00214FF40050CFE754
:10C4C00008BD00BF000C004000140040002C0140DB
:10C4D000038810B503F08F0303804C88CB88028853
:10C4E000234313439BB203808B8883850B8803858A
:10C4F000054B984203D003F50063984201D10B7AB3
:10C5000003860123838210BD002C0140038C30B5CB
:10C5100023F001031B041B0C0384038C8288048B0F
:10C520000D8824F070042404240C23F002032C430F
:10C530001B040D891B0C2B434D8892B22B43CD88D5
:10C5400085860D4DA84203D005F50065A8420FD1A0
:10C550004D8923F008032B438D8823F0040322F434
:10C5600040722B4352048D89520CC9892A430A43D5
:10C5700082800483038430BD002C0140038C70B59D
:10C5800023F010031B041B0C0384038C8488028B90
:10C590000D8822F4E0421204120C42EA05224E8871
:10C5A0000D8923F020031B0435431B0C43EA0513BC
:10C5B000CD88A4B20587114D92B2A8429BB203D098
:10C5C00005F50065A84215D14D8923F0800343EAA3
:10C5D00005134FF6BF751D408B8824F4406445EA6F
:10C5E00003138D89C9896404640C294344EA8104D6
:10C5F0009BB2A4B284800283038470BD002C0140EE
:10C60000038C70B523F480731B041B0C0384038C10
:10C610008288848B0D8824F070042404240C4E88B6
:10C620002C4323F400730D891B0435431B0C43EA90
:10C630000523CD8892B28587104D9BB2A84203D0C6
:10C6400005F50065A84215D14D8923F4006343EA3E
:10C6500005234FF6FF351D408B8822F4405245EAF2
:10C6600003238D89C9895204520C294342EA0112DD
:10C670009BB292B282808483038470BD002C0140FF
:10C68000038C70B523F480531B041B0C0384038CB0
:10C690008488828B0D8822F4E0421204120C42EA54
:10C6A00005224E880D8923F400531B0435431B0CCF
:10C6B00043EA0533CD88A4B2A0F84050094D92B2A8
:10C6C000A8429BB203D005F50065A84205D189892F
:10C6D000C4F30D0444EA8114A4B2848082830384E9
:10C6E00070BD00BF002C01404A880B8813438A8824
:10C6F0001343CA8813430A8913434A8913438A8917
:10C7000013439BB2A0F8443070474FF6FF73838009
:10C7100000230380C380438003727047002303809B
:10C7200043808380C380038143818381C3817047B9
:10C7300000230122038043808280C38003817047ED
:10C740000023038043808380C380038143818381EE
:10C750007047038821B19BB243F001030380704707
:10C7600023F001039B059B0DF8E7B0F8443039B185
:10C770006FEA43436FEA53439BB2A0F844307047DB
:10C78000C3F30E03F9E7818270470A43A0F84820FB
:10C79000704783899BB212B119438181704723EAA4
:10C7A0000101FAE7FFF7F5BF038923F007031B0434
:10C7B0001B0C03817047038923F070031B041B0CBF
:10C7C0001943018103899BB243F00703038170473A
:10C7D00038B50D46602D114604464FF001020ED1CA
:10C7E000FFF7EDFD218921F070010904090C2943AF
:10C7F000218123899BB243F00703238138BDFFF7D2
:10C80000C3FDEFE710B5048942EA0323E4B21943FC
:10C810000C43A4B2048110BD10B5FFF7F3FF0389E8
:10C8200023F077031B041B0C43F07703038110BD37
:10C8300010B5FFF7E7FF03899BB243F48043038100
:10C8400010BD018582827047038823F070039B0529
:10C850009B0D194301807047038923F070031B046B
:10C860001B0C19430181704770B50689048B058C38
:10C8700024F4407424F0030425F0220526F0070672
:10C8800024042D043604240C2D0C42EA0313360C28
:10C8900044F480741D43314344F00104ADB201817E
:10C8A0000483058470BD038B23F070031B041B0CF1
:10C8B000194301837047038B23F4E0431B041B0CD3
:10C8C00043EA012189B201837047838B23F070030F
:10C8D0001B041B0C194381837047838B23F4E043B3
:10C8E0001B041B0C43EA012189B281837047038832
:10C8F00021B19BB243F080030380704723F0800393
:10C900009B059B0DF8E7838821B19BB243F004039C
:10C910008380704723F004031B041B0CF8E7838813
:10C9200021B19BB243F008038380704723F00803D2
:10C930001B041B0CF8E7838821B19BB243F0010371
:10C940008380704723F001031B041B0CF8E7038B63
:10C9500023F008031B041B0C194301837047038B4E
:10C9600023F400631B041B0C43EA012189B20183F9
:10C970007047838B23F008031B041B0C194381832E
:10C980007047838B23F400631B041B0C43EA0121D3
:10C9900089B281837047038B23F004031B041B0CB3
:10C9A000194301837047038B23F480631B041B0C22
:10C9B00043EA012189B201837047838B23F004038A
:10C9C0001B041B0C194381837047838B23F4806302
:10C9D0001B041B0C43EA012189B281837047038B3E
:10C9E00023F080031B041B0C194301837047038B46
:10C9F000C3F30E0343EA012189B201837047838B9D
:10CA000023F080031B041B0C194381837047838B25
:10CA1000C3F30E0343EA012189B281837047038C7B
:10CA200023F002031B041B0C194301847047038C81
:10CA300023F008031B041B0C194301847047038C6B
:10CA400023F020031B041B0C43EA011189B201846B
:10CA50007047038C23F080031B041B0C43EA011175
:10CA600089B201847047038C23F400731B041B0CF0
:10CA700043EA012189B201847047038C23F40063E7
:10CA80001B041B0C43EA012189B201847047038C0B
:10CA900023F400531B041B0C43EA013189B20184C7
:10CAA000704710B50124038C8C409BB223EA040329
:10CAB0000384038C02FA01F1194389B2018410BD89
:10CAC00010B50424038C8C409BB223EA0403038436
:10CAD000038C02FA01F1194389B2018410BD10B52B
:10CAE0000124038C8C409BB223EA0403038421F0CD
:10CAF0000803183053B94908435823F070031B0446
:10CB00001B0C435043581A43425010BD0439C1F323
:10CB10004E014358120223F4E0431B041B0C435004
:10CB2000435892B2EFE7038821B19BB243F002036E
:10CB30000380704723F002039B059B0DF8E70388F1
:10CB400021B19BB243F004030380704723F0040338
:10CB50009B059B0DF8E7838821B19BB243F08003CE
:10CB60008380704723F080031B041B0CF8E70388C5
:10CB700023F008039B059B0D038003889BB2194398
:10CB800001807047838823F070031B041B0C838093
:10CB900083889BB2194381807047038923F0070380
:10CBA0001B041B0C038103899BB21943018170474D
:10CBB000038923F080031B041B0C038103899BB2B0
:10CBC0001943018170478184704781857047818650
:10CBD00070470187704781877047A0F84010704701
:10CBE000038B23F00C031B041B0C0383038B9BB2EE
:10CBF000194301837047038B23F440631B041B0C10
:10CC00000383038B9BB243EA012189B201837047FE
:10CC1000F8B50C464988A2880029B4F800E00CBF9A
:10CC200002260026012A0CBF022701272389BEF114
:10CC3000000F0ED1FFF7A8FBE188FFF7D1FF3146C7
:10CC400023893A46FFF7BBFBE188BDE8F840FFF7D0
:10CC5000D2BFFFF7B4FBE188FFF7CDFF3146238950
:10CC60003A46FFF791FBE188BDE8F840FFF7B8BF0F
:10CC7000838B23F00C031B041B0C8383838B9BB2DD
:10CC8000194381837047838B23F440631B041B0C7F
:10CC90008383838B9BB243EA012189B281837047EE
:10CCA000F8B50E880D460B898A88498836B9FFF792
:10CCB0006BFBE988BDE8F840FFF792BF042E06D170
:10CCC000FFF77DFBE988BDE8F840FFF794BF082E29
:10CCD000EE88058C1CD125F480752D042D0C05845F
:10CCE000878B058CBFB227F0F307ADB23A4342EA17
:10CCF000031225F4007343F4807343EA01239BB2CB
:10CD000092B2828331460384BDE8F840FFF7B0BF9A
:10CD100025F480552D042D0C0584878B058C1B0371
:10CD2000ADB227F4407743EA02223F0525F40053D1
:10CD30003F0D43F480533A4343EA01339BB292B22E
:10CD4000828331460384BDE8F840FFF79CBF038827
:10CD5000DBB2038003889BB2194301807047808E49
:10CD600080B27047008F80B27047808F80B270476A
:10CD7000B0F8400080B27047808C80B27047008D60
:10CD800080B27047038A194214BF01200020704707
:10CD9000C94389B201827047038A828911EA03007C
:10CDA00092B203D0114214BF012000207047C94342
:10CDB00089B20182704700BF08B5244B984231D038
:10CDC00008D8A3F50063984217D003F58063984212
:10CDD0001FD008BD1E4B98422DD003F568439842E2
:10CDE00032D101214FF48040FFF79EF8BDE80840A2
:10CDF00000214FF48040FFF797B801214FF4003035
:10CE0000FFF79EF800214FF40030BDE80840FFF71F
:10CE100097B801214FF48020FFF792F800214FF4DA
:10CE20008020F2E701214FF40020FFF789F800216C
:10CE30004FF40020E9E701214FF48010FFF780F85C
:10CE400000214FF48010E0E708BD00BF004C004017
:10CE50000050004030B50446038ACA889BB223F4D0
:10CE600040531343038283898A8823F4B05323F009
:10CE70000C031B041B0C13430A8987B013434A8914
:10CE80000D4613439BB28381838A8A899BB223F424
:10CE900040731343838201A8FEF7E0FF039B049ACB
:10CEA0000D498C4218BF1A46192353432A68920031
:10CEB000B3FBF2F36422B3FBF2F102FB11331B016B
:10CEC0003233B3FBF2F303F00F0343EA01139BB2D7
:10CED000238107B030BD00BF003801404FF4165326
:10CEE0000C220360002342818380C38003818381FD
:10CEF00070470B8810B54C88028A23438C88C988F8
:10CF000092B223430B4322F4706213439BB2038219
:10CF100010BD0023038043808380C38070478389D2
:10CF200021B19BB243F400538381704723F4005333
:10CF30001B041B0CF8E701F01F0310B5C1F34214EA
:10CF40000121012C01FA03F105D10C3003683AB13B
:10CF50001943016010BD022C0CBF10301430F5E7EE
:10CF600023EA0101F5E7838A9BB212B1194381825A
:10CF7000704723EA0101FAE7038A23F00F031B0439
:10CF80001B0C0382038A9BB2194301827047838979
:10CF900023F400631B041B0C838183899BB2194318
:10CFA00081817047838921B19BB243F00203838161
:10CFB000704723F002031B041B0CF8E7038A23F0DD
:10CFC00020031B041B0C0382038A9BB219430182BA
:10CFD0007047038A21B19BB243F4804303827047B8
:10CFE00023F480431B041B0CF8E7C1F30801818084
:10CFF00070478088C0F30800704783899BB243F074
:10D00000010383817047038BDBB20383038B9BB2E5
:10D0100043EA012101837047038B03F47F430383B9
:10D02000038B9BB2194301837047838A21B19BB262
:10D0300043F020038382704723F020031B041B0C62
:10D04000F8E7838A21B19BB243F0100383827047D3
:10D0500023F010031B041B0CF8E7838A21B19BB259
:10D0600043F008038382704723F008031B041B0C62
:10D07000F8E7838A23F004031B041B0C8382838A52
:10D080009BB2194381827047838A21B19BB243F0DE
:10D0900002038382704723F002031B041B0CF8E792
:10D0A0000388194214BF012000207047C94389B288
:10D0B000018070470123C1F3421210B5012A01F02B
:10D0C0001F0403FA04F30ED1828992B2134002883E
:10D0D00092B26BB10123090A03FA01F10A4214BFAB
:10D0E0001846002010BD022A0CBF028A828AECE793
:10D0F000184610BD0B0A01219940C94389B201802D
:10D10000704700BF684620F007018D4601B50C4A04
:10D110000C4B0D498B420AD300210C4B0C4A934215
:10D120000AD302F0ADF9BDE801408546704752F8D8
:10D13000040F43F8040BEDE743F8041BEFE700BFCF
:10D14000ECFF0008000000206405002068050020B6
:10D150001811002010B5064C18B9012223681A8254
:10D1600010BD044B1B681B68984720680A3010BD2F
:10D17000C41000208010002010B5064C18B9012200
:10D1800023681A8210BD044B1B689B68984720686F
:10D190000C3010BDC41000208010002010B5204BB2
:10D1A00018B902221B681A8210BD00201D491C6894
:10D1B000088023780A4613F07F0313D1637A990617
:10D1C00044BF0221117013F0400F137814BF23F0F5
:10D1D000010343F001031370134B1B681B6998474D
:10D1E000104810BD012B18D0022B17D1617901F026
:10D1F0000F039B0003F1804303F5B84311F0800F48
:10D200001B6805D003F03003102BE5D10123E2E7C2
:10D2100003F44053B3F5805FF7E7084610BD00BF45
:10D22000C410002010110020801000202DE9F843C8
:10D23000234FDFF8A0803D682C8AD4B92E7A042EC3
:10D2400017D120490B78012B0ED11F4B1A681F4BA9
:10D2500092B213445B001C6030230C70A8F80030BD
:10D260003B681E72BDE8F88310230726A8F800303B
:10D27000F6E7AB8A9C4294BF042602269C4228BF54
:10D280001C46AB69204698478146002000F0A6FE68
:10D2900022460146484600F06BFC2146002000F083
:10D2A0000DFE2B8A4FF440521B1B2B826B8A1C44B1
:10D2B0003023A8F80030064B6C821A80D0E700BFFC
:10D2C000C4100020F0090020505C00400230002013
:10D2D000121100201411002010B50A4B0A491B68D6
:10D2E0004978DA7891420AD3997841B99C8834B95F
:10D2F0009A72064B1B685B689847204610BD022057
:10D3000010BD00BFC4100020D800002080100020F5
:10D3100038B50F4A0F4D12682B689269D978587941
:10D3200090472B6804469A7A7AB170B91A7962B933
:10D330009B7853B9084B1B68DB6898472B685A7970
:10D34000DA72DA781A73204638BD0224FBE700BF90
:10D350005C100020C41000208010002038B52D4B38
:10D360001B68187810F07F0004D15A7A22F020024E
:10D370005A7238BD02284BD15A88002A49D11A79ED
:10D38000002A46D15979244D21F08000840004F10F
:10D39000804202F5B842126849B22D780029B4BF24
:10D3A00002F0300202F44052A84231D282B39B7A9A
:10D3B00073B304F1804404F5B8440029236811DAFA
:10D3C00003F03003102B07D1C4B2204600F04BFD10
:10D3D0003021204600F04EFC104B1B685B699847DB
:10D3E000002038BD03F44053B3F5805FF4D10C4DF9
:10D3F00058B90C4B93F82C1000F081FD23682B409A
:10D400009BB283F440532360E6E700F019FDF5E793
:10D41000022038BDC4100020D80000208010002059
:10D420008FBFFFFF5000002038B51D4B1D4D186801
:10D430002D78417921F08004A30003F1804202F5A8
:10D44000B842126849B20029B4BF02F0300202F4B7
:10D450004052AC4221D24488FCB9F2B1827AE2B1A6
:10D4600003F1804303F5B8431A680029B5BF22F4DD
:10D47000E04222F4804222F0400222F07002B5BF66
:10D4800092B292B282F0100282F480521A60064B7D
:10D490001B689B699847002038BD022038BD00BF3B
:10D4A000C4100020D80000208010002008B5064BD2
:10D4B0001A68537A43F020035372044B1B68DB69EC
:10D4C0009847002008BD00BFC41000208010002035
:10D4D000054B10B51C68628A18B98B889B1A238289
:10D4E00010BD0868104410BDC410002008B50B4BD7
:10D4F000002093F82C1000F002FD094B1B68187AED
:10D50000082806D14FF48052064B1A801022064B91
:10D510001A80A0F109035842584108BD500000206C
:10D52000C41000201211002014110020F7B5984CEF
:10D53000984E276832683B7A092B19D0964B92B2E5
:10D5400013445B001D886D0005F1804505F5C0455D
:10D550002B783B706B787B70A88800F06DFE78802C
:10D560002889276800F068FEB880AA892368DA80D5
:10D57000012223681A72DA885D78002A63D11A784A
:10D5800012F07F024CD1092D03D1FFF7A5FEB0B1F7
:10D5900026E0052D1FD193F90320002A06DA08237F
:10D5A00022681372FFF7A2FF03B0F0BD9A78002A39
:10D5B000F5D19A88002AF2D19B7A002BEFD13268FC
:10D5C000764B92B2134400225B001A603022744BF7
:10D5D0001A800623E4E7032D14D1DA78012A08D053
:10D5E000704B28461B685B699847032828D109239C
:10D5F000D6E79A88002AF3D15B7A9806F0D5FFF730
:10D6000055FFC4E7012DEBD1DA78012AE8D19A88D9
:10D61000002AE5D15B7A9906E2D5FFF79FFEB6E7CF
:10D62000012A04D10B2DDBD1FFF772FEAFE7022AEE
:10D63000D6D1012DF1D0032DD2D1FFF7F5FEA6E70B
:10D640000028ACD1BBE7062D14D11A7852065DD163
:10D650009A78544B012A03D11B68DB69EBB955E07A
:10D66000022A02D11B681B6AF8E7032A4ED11B6805
:10D670005B6AF3E7002D55D15988002946D15A68D5
:10D6800022F47F42B2F5003F40D11A7812F07F02B7
:10D6900016D19B88002B39D1434B002522682846A0
:10D6A00055829361984728464FF6FF7123681A8A7E
:10D6B0008A4234D0022801D0002A56D108222FE015
:10D6C000012A0AD1374A5879126892699047E8B915
:10D6D00023689B7A002BDFD118E0022A16D15A79F1
:10D6E000324802F00F018B0003F1804303F5B84389
:10D6F0001B68007812F0800F14BF03F0300303F4AE
:10D700004053814202D212F0700FE3D0254B2268C1
:10D710001B6850781B6998470328C5D123680922E4
:10D720001A723FE7082D04D11B785B06EED1204B1F
:10D73000B3E70A2DEAD11A7802F07F02012AE5D177
:10D740009A7A002AE2D059880029DFD15A6822F457
:10D750007F42B2F5803FD9D1124A58791268926956
:10D7600090470028D2D1134B97E793F90010002976
:10D7700035DAD9880B4C0191019882421CD9019A63
:10D780001A82226892F82C209A82FFF74FFD09E74F
:10D79000C4100020505C0040043000200230002003
:10D7A000141100205C1000209DD10008D80000203A
:10D7B00055D1000879D100088A42E2D2216891F857
:10D7C0002C00824203D20021084A1170D9E792FB53
:10D7D000F0F100FB1122002AD3D10121F4E703224A
:10D7E0001A724FF44052024B1A80DBE6F009002017
:10D7F00012110020F8B52A4D2C68237A032B01D092
:10D80000052B44D1A369268AABB1A6B1A28A964260
:10D8100028BF164630469847238A07469B1B23821B
:10D82000638A00203344638200F0E8FB32460146FD
:10D83000384600F0AFF9238A53B100214FF440522B
:10D84000184B08461A8000F039FB3022164B1A801C
:10D85000A38A228A93422B6809D803221A722B6862
:10D860001B7A2A681372BDE8F840FFF73FBE0AB181
:10D870000522F3E7062119720C4B19680C4B89B28B
:10D880000B445B001A603022074B1A80E7E7072B36
:10D8900003D1084B1B68DB6898470823E1E700BF0A
:10D8A000C41000201211002014110020505C004010
:10D8B000023000205C10002030B5002248F68F7541
:10D8C000094B1C78A24204D3084B40F0800018603A
:10D8D00030BD02F1805303F5B8539B00196829400D
:10D8E000114319600132EDE7D80000204C5C004084
:10D8F00010B5134C23681A7A022A01D0042A09D1E0
:10D90000FFF794FC23681B7A22681372BDE810406D
:10D91000FFF7ECBD062A10D15A78052A09D11A78EA
:10D92000520606D1D878FFF7C7FF064B1B681B6A63
:10D930009847054B1B689B6898470823E4E700BF9E
:10D94000C4100020801000205C100020704700BF31
:10D95000064B074A0749136002221A72064B074A10
:10D960001360074A1B681160184700BF641000204D
:10D97000C4100020B4000020500000205C100020E3
:10D98000801000202DE9F843DFF86481DFF864910E
:10D99000D8F800304F4A99B21B04118001D4BDE879
:10D9A000F88347F6FF73C8F80030138803F00F03BD
:10D9B00089F80030002B62D1474C484E2368484D0F
:10D9C00003F4405333802368464F03F030032B8029
:10D9D00023683B409BB283F400532360236823F405
:10D9E000E04323F040039BB283F0200323601388BD
:10D9F00013F0100F236828D123F4E14323F07003C0
:10DA00001B041B0C2360FFF773FF236832883B4025
:10DA10009BB2D70448BF83F4805396042E4A48BF74
:10DA200083F4005313601368298823F4E04323F040
:10DA300040039BB2CC0648BF83F01003880648BF62
:10DA400083F020031360BDE8F883190601D523682D
:10DA5000D2E71A0508D5236823F070031B051B0DB8
:10DA60002360FFF763FDD0E71B0491D5236823F003
:10DA700070031B051B0D2360FFF7BCFEC5E79A0072
:10DA800002F1804202F5B842146821040AD51168F7
:10DA9000013B21F070010905090D1160124A52F88D
:10DAA0002330984722067FF573AF99F80020930042
:10DAB00003F1804303F5B8431968013A21F4E141C9
:10DAC00021F070010904090C1960084B53F8223049
:10DAD00098475DE75A100020005C004012110020BA
:10DAE000141100208FBFFFFFDC000020F800002091
:10DAF000445C00406010002070B5184D184C194E61
:10DB00002B689AB21B04228000D470BD47F6FF73C5
:10DB10002B60238803F00F039A0002F180423370D8
:10DB200002F5B842116808040BD51168013B21F0D9
:10DB300070010905090D11600B4A52F8233098470E
:10DB4000DEE70906DCD51168013B21F4E14121F053
:10DB500070010904090C1160044AEEE7445C0040BE
:10DB60005A10002060100020DC000020F800002087
:10DB7000002310B501F10051013201F5405152105E
:10DB800049009A4200D110BD30F8024B21F82340E1
:10DB90000133F6E7002310B501F10051013201F520
:10DBA0004051521049009A4200D110BD51F8234013
:10DBB00020F813400133F6E7014B1860704700BFAF
:10DBC000405C0040014B186880B27047405C0040E8
:10DBD000014B1860704700BF445C0040014B18685F
:10DBE00080B27047445C0040014B186880B27047B7
:10DBF000485C0040014B1860704700BF4C5C00401F
:10DC0000014B186880B270474C5C00404FF6F873C7
:10DC1000014A034013607047505C0040014B186894
:10DC200080B27047505C0040800000F1804000F5F9
:10DC3000B84001607047800000F1804000F5B840B6
:10DC4000006880B27047800000F1804000F5B84065
:10DC5000036823F4EC4323F07003194389B2016095
:10DC60007047800000F1804000F5B840006800F483
:10DC7000C0607047800000F1804000F5B840036844
:10DC8000CA0623F4E04323F040039BB248BF83F06D
:10DC900010038A0648BF83F02003036070478000AA
:10DCA00000F1804000F5B8400368CA0423F48043C3
:10DCB00023F070039BB248BF83F480538A0448BFAB
:10DCC00083F4005303607047800000F1804000F54A
:10DCD000B8400129036805D123F480531B041B0CB1
:10DCE000036070470229FCD123F01003F6E780009F
:10DCF00000F1804000F5B840006800F03000704747
:10DD0000800000F1804000F5B840006800F4405009
:10DD10007047800000F1804000F5B840036823F4AC
:10DD2000E04323F040039BB283F03003036070476D
:10DD3000800000F1804000F5B840036823F4804380
:10DD400023F070039BB283F440530360704780005C
:10DD500000F1804000F5B840036823F4E04323F06D
:10DD6000700343F480739BB203607047FFF7EFBF0B
:10DD7000FFF7EDBF800000F1804000F5B840036878
:10DD800023F4E24323F070031B041B0C0360704771
:10DD9000FFF7F0BFFFF7EEBF800000F1804000F515
:10DDA000B840006800F03000A0F11003584258411C
:10DDB0007047800000F1804000F5B840006800F432
:10DDC0004050A0F58053584258417047800000F100
:10DDD000804000F5B840036823F070031B051B0D5D
:10DDE00003607047800000F1804000F5B840036890
:10DDF00023F4E14323F070031B041B0C0360704702
:10DE0000800000F1804000F5B840036823F4E0434F
:10DE100023F070031B041B0C43F480430360704722
:10DE2000800000F1804000F5B840036823F4E0432F
:10DE300023F070031B041B0C43F040030360704786
:10DE4000800000F1804000F5B84003685B0409D50C
:10DE5000036823F4E04323F070031B041B0C43F41A
:10DE6000804303607047800000F1804000F5B840B7
:10DE700003685B0609D5036823F4E04323F07003CD
:10DE80001B041B0C43F0400303607047800000F14B
:10DE9000804000F5B840036823F4E04323F07003AA
:10DEA0001B041B0C194301607047800000F1804087
:10DEB00000F5B840006800F00F007047044B1B6885
:10DEC0009BB203EBC000034B03445B001960704737
:10DED000505C0040023000203E290AD94B09C90697
:10DEE00004BF03F1FF339BB29B0243F40043036082
:10DEF00070474B08CA0748BF01339B02F7E70E4B38
:10DF00000E4A1B683E299BB203EBC00002444FEA55
:10DF100042020AD94B09C80604BF03F1FF339BB282
:10DF20009B0243F40043136070474B08C90748BF86
:10DF300001339B02F7E700BF505C00400630002031
:10DF400010B50B4CC000236849089BB2034403F191
:10DF5000005303F540535B004900196023685208E1
:10DF60009BB21844034B520003445B001A6010BD7F
:10DF7000505C004004300020064B49081B684900F3
:10DF80009BB203EBC00000F1005000F54050400090
:10DF900001607047505C0040FFF7EEBF054B490839
:10DFA0001B6849009BB203EBC000034B03445B00BA
:10DFB00019607047505C004004300020FFF7EEBF4E
:10DFC000054B1B689BB203EBC00000F1005000F54D
:10DFD0004050400000887047505C0040FFF7F0BFA1
:10DFE000044B1B689BB203EBC000034B03445B0074
:10DFF00018887047505C004004300020FFF7F0BFE5
:10E00000012910B52BD1254CC0002168244B89B2C1
:10E0100001440B443E2A4FEA430119D9530912F037
:10E020001F0F04BF03F1FF339BB29B0243F4004375
:10E030000B6023681B499BB2184401443E2A4FEAF7
:10E0400041011FD85308D20748BF01339B0222E089
:10E05000530812F0010F18BF01339B02E8E70229B1
:10E060001BD10E4CC00021680D4B89B201440B44FA
:10E070005B001A6023689BB218440A4B03445B00A0
:10E080001A6010BD5309D00604BF03F1FF339BB2E1
:10E090009B0243F400430B6010BD10BD505C004078
:10E0A000023000200630002001291BD1134B1449F7
:10E0B0001B683E2A9BB203EBC00001444FEA4101BA
:10E0C0000AD95309D00604BF03F1FF339BB29B0268
:10E0D00043F400430B6070475308D20748BF013335
:10E0E0009B02F7E7022908D1044B1B689BB203EBA4
:10E0F000C000034B03445B001A607047505C004053
:10E100000230002001291BD1134B14491B683E2A01
:10E110009BB203EBC00001444FEA41010AD9530905
:10E12000D00604BF03F1FF339BB29B0243F40043CC
:10E130000B6070475308D20748BF01339B02F7E7D3
:10E14000022908D1044B1B689BB203EBC000034BB0
:10E1500003445B001A607047505C004006300020AA
:10E16000054B1B689BB203EBC000044B03445B00F0
:10E170001868C0F309007047505C0040023000206E
:10E18000FFF7EEBF054B1B689BB203EBC000044BCF
:10E1900003445B001868C0F309007047505C0040FE
:10E1A00006300020FFF7EEBF0D49C0000B689BB2A0
:10E1B000C2180C4B13445B001B6813F47C4F0DD149
:10E1C0000B689BB21844084B03445B001B68C3F305
:10E1D0000903002B14BF0220002070470120704764
:10E1E000505C0040063000200230002001290FD191
:10E1F000800000F1804000F5B840036823F4E0435C
:10E2000023F070031B041B0C43F0400303607047B2
:10E210000229FCD1800000F1804000F5B84003687D
:10E2200023F4E04323F070031B041B0C43F48043EE
:10E23000ECE741EA00207047C3B2000A40EA03203D
:10E24000704700BF81F0004102E000BF83F000434F
:10E2500030B54FEA41044FEA430594EA050F08BF81
:10E2600090EA020F1FBF54EA000C55EA020C7FEA45
:10E27000645C7FEA655C00F0E2804FEA5454D4EBC2
:10E280005555B8BF6D420CDD2C4480EA020281EA8C
:10E29000030382EA000083EA010180EA020281EAC4
:10E2A0000303362D88BF30BD11F0004F4FEA013116
:10E2B0004FF4801C4CEA113102D0404261EB410125
:10E2C00013F0004F4FEA03334CEA133302D05242AB
:10E2D00063EB430394EA050F00F0A780A4F1010467
:10E2E000D5F1200E0DDB02FA0EFC22FA05F28018A1
:10E2F00041F1000103FA0EF2801843FA05F3594187
:10E300000EE0A5F120050EF1200E012A03FA0EFC05
:10E3100028BF4CF0020C43FA05F3C01851EBE3712F
:10E3200001F0004507D54FF0000EDCF1000C7EEB4C
:10E3300000006EEB0101B1F5801F1BD3B1F5001F8A
:10E340000CD349085FEA30004FEA3C0C04F10104A9
:10E350004FEA445212F5800F80F09A80BCF1004FD2
:10E3600008BF5FEA500C50F1000041EB045141EA54
:10E37000050130BD5FEA4C0C404141EB010111F455
:10E38000801FA4F10104E9D191F0000F04BF014600
:10E390000020B1FA81F308BF2033A3F10B03B3F1DE
:10E3A00020020CDA0C3208DD02F1140CC2F10C026E
:10E3B00001FA0CF021FA02F10CE002F11402D8BFCC
:10E3C000C2F1200C01FA02F120FA0CFCDCBF41EA98
:10E3D0000C019040E41AA2BF01EB0451294330BD67
:10E3E0006FEA04041F3C1CDA0C340EDC04F1140444
:10E3F000C4F1200220FA04F001FA02F340EA03001B
:10E4000021FA04F345EA030130BDC4F10C04C4F160
:10E41000200220FA02F001FA04F340EA0300294640
:10E4200030BD21FA04F0294630BD94F0000F83F48A
:10E43000801306BF81F480110134013D4EE77FEA6D
:10E44000645C18BF7FEA655C29D094EA050F08BFB9
:10E4500090EA020F05D054EA000C04BF194610469A
:10E4600030BD91EA030F1EBF0021002030BD5FEADE
:10E47000545C05D14000494128BF41F0004130BD06
:10E4800014F580043CBF01F5801130BD01F000455A
:10E4900045F0FE4141F470014FF0000030BD7FEACD
:10E4A000645C1ABF194610467FEA655C1CBF0B46C8
:10E4B000024650EA013406BF52EA033591EA030FDF
:10E4C00041F4002130BD00BF90F0000F04BF0021D7
:10E4D000704730B54FF4806404F132044FF000050A
:10E4E0004FF0000150E700BF90F0000F04BF002183
:10E4F000704730B54FF4806404F1320410F00045E9
:10E5000048BF40424FF000013EE700BF42004FEAE3
:10E51000E2014FEA31014FEA02701FBF12F07F4360
:10E5200093F07F4F81F06051704792F0000F14BF5D
:10E5300093F07F4F704730B54FF4607401F00045A1
:10E5400021F0004120E700BF50EA010208BF7047F8
:10E5500030B54FF000050AE050EA010208BF7047ED
:10E5600030B511F0004502D5404261EB41014FF456
:10E57000806404F132045FEA915C3FF4DCAE4FF05A
:10E5800003025FEADC0C18BF03325FEADC0C18BF41
:10E59000033202EBDC02C2F1200300FA03FC20FA92
:10E5A00002F001FA03FE40EA0E0021FA02F11444DF
:10E5B000C1E600BF70B54FF0FF0C4CF4E06C1CEAF4
:10E5C00011541DBF1CEA135594EA0C0F95EA0C0F69
:10E5D00000F0DEF82C4481EA030621EA4C5123EADC
:10E5E0004C5350EA013518BF52EA033541F480110B
:10E5F00043F4801338D0A0FB02CE4FF00005E1FBBE
:10E6000002E506F00042E0FB03E54FF00006E1FB07
:10E6100003569CF0000F18BF4EF0010EA4F1FF044A
:10E62000B6F5007F64F5407404D25FEA4E0E6D418A
:10E6300046EB060642EAC62141EA55514FEAC5209B
:10E6400040EA5E504FEACE2EB4F1FD0C88BFBCF517
:10E65000E06F1ED8BEF1004F08BF5FEA500E50F1C8
:10E66000000041EB045170BD06F0004646EA01018E
:10E6700040EA020081EA0301B4EB5C04C2BFD4EBC0
:10E680000C0541EA045170BD41F480114FF0000EB9
:10E69000013C00F3AB8014F1360FDEBF002001F027
:10E6A000004170BDC4F10004203C35DA0C341BDCA1
:10E6B00004F11404C4F1200500FA05F320FA04F073
:10E6C00001FA05F240EA020001F0004221F00041A7
:10E6D00010EBD37021FA04F642EB06015EEA430E1A
:10E6E00008BF20EAD37070BDC4F10C04C4F120054A
:10E6F00000FA04F320FA05F001FA04F240EA0200FD
:10E7000001F0004110EBD37041F100015EEA430ECD
:10E7100008BF20EAD37070BDC4F1200500FA05F2ED
:10E720004EEA020E20FA04F301FA05F243EA02036C
:10E7300021FA04F001F0004121FA04F220EA02007B
:10E7400000EBD3705EEA430E08BF20EAD37070BDC1
:10E7500094F0000F0FD101F00046400041EB0101A1
:10E7600011F4801F08BF013CF7D041EA060195F083
:10E77000000F18BF704703F00046520043EB03033D
:10E7800013F4801F08BF013DF7D043EA060370472A
:10E7900094EA0C0F0CEA135518BF95EA0C0F0CD035
:10E7A00050EA410618BF52EA4306D1D181EA03017B
:10E7B00001F000414FF0000070BD50EA410606BF75
:10E7C0001046194652EA430619D094EA0C0F02D1BA
:10E7D00050EA013613D195EA0C0F05D152EA0336FF
:10E7E0001CBF104619460AD181EA030101F000411D
:10E7F00041F0FE4141F470014FF0000070BD41F066
:10E80000FE4141F4780170BD70B54FF0FF0C4CF43F
:10E81000E06C1CEA11541DBF1CEA135594EA0C0F5E
:10E8200095EA0C0F00F0A7F8A4EB050481EA030EAB
:10E8300052EA03354FEA013100F088804FEA033392
:10E840004FF0805545EA131343EA12634FEA022260
:10E8500045EA111545EA10654FEA00260EF0004121
:10E860009D4208BF964244F1FD0404F5407402D273
:10E870005B084FEA3202B61A65EB03055B084FEA04
:10E8800032024FF480104FF4002CB6EB020E75EB01
:10E89000030E22BFB61A754640EA0C005B084FEA29
:10E8A0003202B6EB020E75EB030E22BFB61A7546A6
:10E8B00040EA5C005B084FEA3202B6EB020E75EBF1
:10E8C000030E22BFB61A754640EA9C005B084FEA69
:10E8D0003202B6EB020E75EB030E22BFB61A754676
:10E8E00040EADC0055EA060E18D04FEA051545EA65
:10E8F00016754FEA06164FEAC30343EA52734FEA0E
:10E90000C2025FEA1C1CC0D111F4801F0BD141EA86
:10E9100000014FF000004FF0004CB6E711F4801FEB
:10E9200004BF01430020B4F1FD0C88BFBCF5E06FCB
:10E930003FF6AFAEB5EB030C04BFB6EB020C5FEADB
:10E94000500C50F1000041EB045170BD0EF0004E30
:10E950004EEA113114EB5C04C2BFD4EB0C0541EA62
:10E96000045170BD41F480114FF0000E013C90E65F
:10E9700045EA060E8DE60CEA135594EA0C0F08BF23
:10E9800095EA0C0F3FF43BAF94EA0C0F0AD150EA22
:10E9900001347FF434AF95EA0C0F7FF425AF1046B5
:10E9A00019462CE795EA0C0F06D152EA03353FF4DD
:10E9B000FDAE1046194622E750EA410618BF52EA5A
:10E9C00043067FF4C5AE50EA41047FF40DAF52EA2E
:10E9D00043057FF4EBAE12E74FF0FF3C06E000BFCB
:10E9E0004FF0010C02E000BF4FF0010C4DF804CDD8
:10E9F0004FEA410C7FEA6C5C4FEA430C18BF7FEA98
:10EA00006C5C1BD001B050EA410C0CBF52EA430CC5
:10EA100091EA030F02BF90EA020F0020704710F145
:10EA2000000F91EA030F58BF994208BF90422CBFD4
:10EA3000D8176FEAE37040F0010070474FEA410CCD
:10EA40007FEA6C5C02D150EA013C07D14FEA430CEB
:10EA50007FEA6C5CD6D152EA033CD3D05DF8040B5C
:10EA6000704700BF8446104662468C46194663468E
:10EA700000E000BF01B5FFF7B7FF002848BF10F165
:10EA8000000F01BD4DF808EDFFF7F4FF0CBF0120AA
:10EA900000205DF808FB00BF4DF808EDFFF7EAFF26
:10EAA00034BF012000205DF808FB00BF4DF808EDE1
:10EAB000FFF7E0FF94BF012000205DF808FB00BFD6
:10EAC0004DF808EDFFF7CEFF94BF012000205DF860
:10EAD00008FB00BF4DF808EDFFF7C4FF34BF01206D
:10EAE00000205DF808FB00BF4FEA410C7FEA6C5C38
:10EAF00002D150EA013C0AD14FEA430C7FEA6C5C38
:10EB000002D152EA033C02D14FF0000070474FF0AF
:10EB1000010070474FEA410212F5001215D211D5DB
:10EB20006FF47873B3EB625212D94FEAC12343F00A
:10EB3000004343EA505311F0004F23FA02F018BF8C
:10EB4000404270474FF00000704750EA013005D155
:10EB500011F0004008BF6FF0004070474FF0000018
:10EB6000704700BF4FEA4102B2F1E04324BFB3F562
:10EB7000001CDCF1FE5C0DD901F0004C4FEAC00234
:10EB80004CEA5070B2F1004F40EB830008BF20F018
:10EB90000100704711F0804F21D113F13872BCBFD2
:10EBA00001F00040704741F480114FEA5252C2F127
:10EBB0001802C2F1200C10FA0CF320FA02F018BF70
:10EBC00040F001004FEAC1234FEAD32303FA0CFCC3
:10EBD00040EA0C0023FA02F34FEA4303CCE77FEA52
:10EBE000625307D150EA01331EBF4FF0FE4040F49C
:10EBF0004000704701F0004040F0FE4040F400004B
:10EC0000704700BF80F0004002E000BF81F000418B
:10EC100042001FBF5FEA410392EA030F7FEA226CC2
:10EC20007FEA236C6AD04FEA1262D2EB1363C1BF52
:10EC3000D218414048404140B8BF5B42192B88BFC1
:10EC4000704710F0004F40F4000020F07F4018BFE4
:10EC5000404211F0004F41F4000121F07F4118BF04
:10EC6000494292EA030F3FD0A2F1010241FA03FCAC
:10EC700010EB0C00C3F1200301FA03F100F0004394
:10EC800002D5494260EB4000B0F5000F13D3B0F15C
:10EC9000807F06D340084FEA310102F10102FE2ACB
:10ECA00051D2B1F1004F40EBC25008BF20F001003B
:10ECB00040EA03007047490040EB000010F4000FE9
:10ECC000A2F10102EDD1B0FA80FCACF1080CB2EB7C
:10ECD0000C0200FA0CF0AABF00EBC25052421843DB
:10ECE000BCBFD0401843704792F0000F81F4000180
:10ECF00006BF80F400000132013BB5E74FEA410353
:10ED00007FEA226C18BF7FEA236C21D092EA030FBE
:10ED100004D092F0000F08BF0846704790EA010F38
:10ED20001CBF0020704712F07F4F04D1400028BF65
:10ED300040F00040704712F100723CBF00F5000047
:10ED4000704700F0004343F0FE4040F4000070477D
:10ED50007FEA226216BF08467FEA23630146420229
:10ED600006BF5FEA412390EA010F40F4800070473C
:10ED70004FF0000304E000BF10F0004348BF4042E2
:10ED80005FEA000C08BF704743F0964301464FF01E
:10ED900000001CE050EA010208BF70474FF000037A
:10EDA0000AE000BF50EA010208BF704711F00043BB
:10EDB00002D5404261EB41015FEA010C02BF84468B
:10EDC0000146002043F0B64308BFA3F18053A3F5EA
:10EDD0000003BCFA8CF2083AA3EBC25310DB01FA31
:10EDE00002FC634400FA02FCC2F12002BCF1004FB5
:10EDF00020FA02F243EB020008BF20F00100704746
:10EE000002F1200201FA02FCC2F1200250EA4C0099
:10EE100021FA02F243EB020008BF20EADC707047DF
:10EE20004FF0FF0C1CEAD0521EBF1CEAD15392EAED
:10EE30000C0F93EA0C0F6FD01A4480EA010C4002C9
:10EE400018BF5FEA41211ED04FF0006343EA501023
:10EE500043EA5111A0FB01310CF00040B1F5000F65
:10EE60003EBF490041EAD3715B0040EA010062F114
:10EE70007F02FD2A1DD8B3F1004F40EBC25008BFFE
:10EE800020F00100704790F0000F0CF0004C08BF1C
:10EE900049024CEA502040EA51207F3AC2BFD2F1E9
:10EEA000FF0340EAC250704740F400004FF00003F7
:10EEB000013A5DDC12F1190FDCBF00F00040704731
:10EEC000C2F10002410021FA02F1C2F1200200FA6F
:10EED00002FC5FEA310040F1000053EA4C0308BF36
:10EEE00020EADC70704792F0000F00F0004C02BF87
:10EEF000400010F4000F013AF9D040EA0C0093F002
:10EF0000000F01F0004C02BF490011F4000F013B5B
:10EF1000F9D041EA0C018FE70CEAD15392EA0C0FC9
:10EF200018BF93EA0C0F0AD030F0004C18BF31F034
:10EF3000004CD8D180EA010000F00040704790F00A
:10EF4000000F17BF90F0004F084691F0000F91F0AE
:10EF5000004F14D092EA0C0F01D142020FD193EA74
:10EF60000C0F03D14B0218BF084608D180EA0100FC
:10EF700000F0004040F0FE4040F40000704740F0D8
:10EF8000FE4040F4400070474FF0FF0C1CEAD052A6
:10EF90001EBF1CEAD15392EA0C0F93EA0C0F69D002
:10EFA000A2EB030280EA010C49024FEA402037D06D
:10EFB0004FF0805343EA111143EA10130CF0004064
:10EFC0008B4238BF5B0042F17D024FF4000C8B4254
:10EFD00024BF5B1A40EA0C00B3EB510F24BFA3EB34
:10EFE000510340EA5C00B3EB910F24BFA3EB910304
:10EFF00040EA9C00B3EBD10F24BFA3EBD10340EA5E
:10F00000DC001B0118BF5FEA1C1CE0D1FD2A3FF6A3
:10F0100050AF8B4240EBC25008BF20F00100704758
:10F020000CF0004C4CEA50207F32C2BFD2F1FF03FB
:10F0300040EAC250704740F400004FF00003013A2C
:10F0400037E792F0000F00F0004C02BF400010F4D0
:10F05000000F013AF9D040EA0C0093F0000F01F0E4
:10F06000004C02BF490011F4000F013BF9D041EA06
:10F070000C0195E70CEAD15392EA0C0F08D1420239
:10F080007FF47DAF93EA0C0F7FF470AF084676E70C
:10F0900093EA0C0F04D14B023FF44CAF08466EE7E5
:10F0A00030F0004C18BF31F0004CCAD130F00042B3
:10F0B0007FF45CAF31F000437FF43CAF5FE700BF0B
:10F0C00042000ED2B2F1FE4F0BD34FF09E03B3EBD2
:10F0D000126209D44FEA002343F0004323FA02F0FE
:10F0E00070474FF00000704712F1610F01D14202EA
:10F0F00002D14FF0FF3070474FF00000704700BF63
:10F100007BB972B90029BEBF00204FF0004106E074
:10F1100008BF00281CBF6FF000414FF0FF3000F027
:10F12000ADB9ADF1080C6DE904CE002909DB002B67
:10F130001ADB00F035F8DDF804E0DDE9022304B065
:10F140007047404261EB4101002B1BDB00F028F8C7
:10F15000DDF804E0DDE9022304B0404261EB410147
:10F16000524263EB43037047524263EB430300F0A8
:10F1700017F8DDF804E0DDE9022304B0404261EB5A
:10F1800041017047524263EB430300F009F8DDF898
:10F1900004E0DDE9022304B0524263EB430370470D
:10F1A0002DE9F0478C460E460446089D002B50D1B1
:10F1B0008A4217466CD9B2FA82FEBEF1000F0BD01C
:10F1C000CEF1200C01FA0EF620FA0CFC02FA0EF732
:10F1D0004CEA060C00FA0EF43A0CBCFBF2F9BBB296
:10F1E00002FB19CC09FB03FA4FEA144848EA0C4623
:10F1F000B2450AD9F61909F1FF3180F02581B245EF
:10F2000040F22281A9F102093E44A6EB0A06B6FBB0
:10F21000F2F002FB106600FB03F3A4B244EA0644DA
:10F22000A34209D9E41900F1FF3280F00B81A34217
:10F2300040F2088102383C440021E41A40EA0940C7
:10F24000002D62D0002324FA0EF42C606B60BDE820
:10F25000F0878B4207D9002D55D0002185E8410069
:10F260000846BDE8F087B3FA83F1002940F08F80AB
:10F27000B34202D3824200F2FC80841A66EB03069A
:10F280000120B446002D40D085E81010BDE8F0877D
:10F2900012B90127B7FBF2F7B7FA87FEBEF1000FEC
:10F2A00035D10121F61B4FEA174C1FFA87F8B6FB40
:10F2B000FCF20CFB126608FB02F0230C43EA064644
:10F2C000B04207D9F61902F1FF3302D2B04200F280
:10F2D000D2801A46361AB6FBFCF00CFB106608FB0F
:10F2E00000F8A3B243EA0644A04507D9E41900F1A7
:10F2F000FF3302D2A04500F2B9801846A4EB0804FF
:10F3000040EA02409CE729462846BDE8F08707FA14
:10F310000EF7CEF1200326FA03F24FEA174CB2FBA8
:10F32000FCF11FFA87F80CFB112206FA0EF620FA00
:10F3300003F301FB08F933431E0C46EA0246B145CC
:10F3400000FA0EF409D9F61901F1FF3280F08C8031
:10F35000B14540F2898002393E44A6EB0906B6FB6E
:10F36000FCF00CFB106200FB08F99EB246EA024674
:10F37000B14507D9F61900F1FF3371D2B1456FD904
:10F3800002383E44A6EB090640EA01418FE7C1F18D
:10F39000200722FA07F88B4048EA030326FA07F40D
:10F3A0004FEA134EB4FBFEF91FFA83FC0EFB19441F
:10F3B0008E4020FA07F809FB0CFA48EA06084FEAE3
:10F3C000184646EA0444A24502FA01F200FA01F6A0
:10F3D00008D9E41809F1FF3044D2A24542D9A9F175
:10F3E00002091C44A4EB0A04B4FBFEF00EFB10441B
:10F3F00000FB0CFC1FFA88F848EA0444A44507D92E
:10F40000E41800F1FF3E29D2A44527D902381C4454
:10F4100040EA0940A0FB0289A4EB0C0CCC45C24693
:10F42000CE4615D312D055B1B6EB0A036CEB0E06DF
:10F4300006FA07F7CB401F43CE402F606E600021D5
:10F44000BDE8F0871046F7E68946DEE64645EAD293
:10F45000B8EB020A69EB030E0138E4E77046D7E720
:10F4600018468FE78146BDE7114676E702383C44EF
:10F4700044E7084606E7023A3E442BE7704700BFE0
:10F480002DE9F3410025694CFCF71EFC4FF4803058
:10F490002570FCF737FCFCF785FD0128064626D1D0
:10F4A0001020FBF717FF2846FCF77AFC2846FCF7EC
:10F4B0008BFC4FF48060FCF77DFC4FF440304FF440
:10F4C000E011FCF74BFC3046FCF752FC3920FCF70E
:10F4D00055FD0028FAD00220FBF7E4FE0220FCF7DD
:10F4E0004DFCFCF755FC0828FBD1012323700121BA
:10F4F0000420FCF701FD4FF48073ADF804300323C2
:10F500008DF80630182301A949488DF80730FCF71B
:10F5100078F90620FCF72CFD01210846FCF7ECFCED
:10F5200001214FF0C050FCF7F3FC424C4FF48041F6
:10F530004FF00060FCF712FB4FF44070FCF766FAE6
:10F540003D4DF4F74DFEF5F771FAF4F719FEF4F7B7
:10F550006FFFF9F7CDFAF9F7ABFAF8F78CFDF4F78E
:10F56000DDFE2078F8F7F8FDE078F8F73BFF2B7820
:10F5700023B92269A1686079F9F76CF82B780BB18F
:10F58000F9F71AFEFAF71FFFF5F7BEF8F7F764FE72
:10F59000F9F776FE294B01275A68294E22F03042AE
:10F5A0005A605A6842F080425A60F9F799FA8046E8
:10F5B000F7F76EFFF9F7CEFEF9F763FEF9F790FA69
:10F5C000A0EB08000028B8BF4042B0F57A7F14DDF8
:10F5D0002B78FBB1B36813F480530BD12B70F9F780
:10F5E0000BFEF9F7D7FDF4F7CBFD2269A16860792E
:10F5F000F9F730F8F9F774FA8046F5F7C1F8F5F73E
:10F6000007F90028D4D0FAF7DEFEF7F725FEF9F760
:10F610004FFECDE7B368DB04ECD5F9F763F92F7043
:10F62000F4F7AEFDF9F7C8FDE4E700BFFC0E0020DB
:10F630000008014008000020A80E00200010014032
:10F64000000C01402DE9F843C1F30A57A7F2FF353A
:10F65000132D0B460446864611DC002D42DB264F57
:10F6600047FA05F501EA050757EA000E1DD101F03A
:10F670000045C2E9000170462946BDE8F883332DF4
:10F680001FDC4FF0FF35A7F2134725FA07F710EA02
:10F69000070C1FD00D4620EA0704C2E900450B46BF
:10F6A0002246FEF7D3FDBDE8F8834FF0000821EABB
:10F6B0000509C2E900894B464246FEF7C7FDBDE891
:10F6C000F883002401F00045C2E9000120462946E4
:10F6D000BDE8F88301F00045C2E900016046294613
:10F6E000BDE8F883002001F0004106460F462046A1
:10F6F0001946C2E90067C0E7FFFF0F0000000000E5
:10F70000C1F30A522DE9F047A2F2FF36132E0B4641
:10F7100004460D4607468846824622DC002E4FDB13
:10F720003D4A42FA06F901EA090202431ED038A313
:10F73000D3E90023FEF78CFD00220023FFF7CAF96E
:10F7400050B1002D04DD4FF4801343FA06F6B044A7
:10F750004FF0000A28EA0905544629462046BDE82C
:10F76000F087332E06DDB6F5806F3DD01946204672
:10F77000BDE8F0874FF0FF39A2F2134229FA02F9EF
:10F7800010EA090FF2D022A3D3E90023FEF760FDAF
:10F7900000220023FFF79EF90028DDD0002D09DDAF
:10F7A000142E2FD00123C6F1340603FA06F63719BA
:10F7B00028BF9844454627EA090A54462946CDE71A
:10F7C00013A3D3E90023FEF743FD00220023FFF734
:10F7D00081F90028C0D0002D0FDB55EA040709D0BD
:10F7E0004FF0000A0D4DB7E702460B46FEF730FD1D
:10F7F0000446BCE7BA463D46AEE74FF0000A4FF07C
:10F800000045A9E705F10108D4E700BFAFF3008088
:10F810009C7500883CE4377EFFFF0F000000F03F3E
:10F82000C1F30A522DE9F843A2F2FF36132E0B461C
:10F8300004460D46884607461DDC002E40DB3C4A48
:10F84000864642FA06F901EA0902024318D036A3B5
:10F85000D3E90023FEF7FCFC00220023FFF73AF96E
:10F8600020B1002D42DB002728EA09053C46294645
:10F870002046BDE8F883332E06DDB6F5806F2FD025
:10F8800019462046BDE8F8834FF0FF39A2F2134233
:10F8900029FA02F910EA090FF2D023A3D3E90023D1
:10F8A000FEF7D6FC00220023FFF714F90028DDD074
:10F8B000002D21DB454627EA09073C462946D7E7C4
:10F8C00019A3D3E90023FEF7C3FC00220023FFF7AE
:10F8D00001F90028CAD0002D19DB00273D46C5E7F5
:10F8E00002460B46FEF7B4FC0446CAE74FF4801309
:10F8F00043FA06F6B044B6E7142E10D00123C6F141
:10F90000340603FA06F6371928BF9844D2E725F0E3
:10F910000042084B224318BF1D460027A6E705F109
:10F920000108C7E7AFF300809C7500883CE4377E90
:10F93000FFFF0F000000F0BF2DE9F0438BB004463D
:10F940000D4600F079F8374B804693F90060894600
:10F95000731C0DD022462B4620462946FFF7C4F8DB
:10F9600030B90022002320462946FFF7B3F820B122
:10F97000404649460BB0BDE8F0832B4B0890CDE9DB
:10F980000245CDE904450193DEB94FF06046274FAB
:10F990002046294600220023CDE90667FFF772F8CA
:10F9A000002837D002230093684600F039FAC8B126
:10F9B000089BE3B9DDE90689404649460BB0BDE83E
:10F9C000F0834FF00008DFF86C90204629460022B3
:10F9D0000023CDE90689FFF755F868B102239E425E
:10F9E0000093E1D100F024FA22230360E0E700F065
:10F9F0001FFA089B0360DDE70123022E00930BD161
:10FA000000F016FA21230360094800F00BFACDE953
:10FA10000601CDE701230093684600F001FA0028B3
:10FA2000F2D1EDE760050020D8FF0008FFFFEFC727
:10FA3000DCFF00080000F0FF2DE9F04FB1F5801F5A
:10FA400085B006460F460B465ADA024621F00044BE
:10FA5000224300F0F8800029C0F27A810022D64BC0
:10FA6000FEF7A8FD0B46D54A064693420F466FF0B7
:10FA7000350C4ADCC3F3130505F5152E0EF6647E2E
:10FA80000EF4801E8EF07F5282F440121C1542EA62
:10FA90000507A4F2FF3464440022C94B30463946BE
:10FAA00004EB1E54FEF7D2FBAB1CC3F31303022B73
:10FAB00082468B464FF0000230DC0023FEF7E2FF67
:10FAC000002800F0C980002C00F04B812046FEF792
:10FAD0000BFDA5A3D3E9002306460F46FEF76AFDFA
:10FAE000A3A3D3E9002304460D4630463946FEF76A
:10FAF00061FD02460B4620462946FEF7A9FB0AE0B7
:10FB0000AE4A4FF0000C9342B4DD32463B463046DD
:10FB10003946FEF79DFB05B0BDE8F08F4FF08043FE
:10FB2000FEF796FB02460B4650465946FEF76CFE22
:10FB3000064620460F46FEF7D7FC3246CDE90001C7
:10FB40003B4630463946CDE90267FEF733FD0246B3
:10FB50000B4680468946FEF72DFD87A3D3E9002397
:10FB600006460F46FEF726FD85A3D3E90023FEF7E0
:10FB70006FFB32463B46FEF71DFD83A3D3E900230E
:10FB8000FEF766FB32463B46FEF714FD80A3D3E941
:10FB90000023FEF75DFB42464B46FEF70BFD7EA3BE
:10FBA000D3E900238046894630463946FEF702FDF8
:10FBB0007BA3D3E90023FEF74BFB32463B46FEF71F
:10FBC000F9FC79A3D3E90023FEF742FB32463B461A
:10FBD000FEF7F0FC0B46024649464046FEF738FB6E
:10FBE000A5F5C223C5F5D725A3F27A4351351D43A8
:10FBF000002D8046894656DD0022724B50465946FC
:10FC0000FEF7D8FC52465B46FEF7D4FC06460F468C
:10FC1000002C68D132463B4640464946FEF718FB69
:10FC2000DDE90223FEF7C6FC02460B4630463946A4
:10FC3000FEF70CFB02460B4650465946FEF706FB04
:10FC400005B0BDE8F08F0022002300205E49FEF7DA
:10FC5000DBFD05B0BDE8F08F55A3D3E90023504686
:10FC60005946FEF7A7FC02460B4600205549FEF711
:10FC7000EDFA524606460F465B4650465946FEF799
:10FC800099FC02460B4630463946FEF793FC064681
:10FC90000F46002C40F09A8002460B4650465946CB
:10FCA000FEF7D4FA37E7002C00F0A4802EA3D3E9A6
:10FCB0000023DDE90001FEF77DFC42464B46044689
:10FCC0000D4650465946FEF7C1FADDE90223FEF71C
:10FCD00071FC27A3D3E9002306460F46DDE90001A6
:10FCE000FEF768FC21E020A3D3E90023DDE9000151
:10FCF000FEF760FC32463B4604460D464046494608
:10FD0000FEF7A6FADDE90223FEF754FC18A3D3E9B7
:10FD1000002380468946DDE90001FEF74BFC0246E0
:10FD20000B4640464946FEF793FA02460B463046DC
:10FD30003946FEF78BFA52465B46FEF787FA0246D3
:10FD40000B4620462946FEF781FA05B0BDE8F08F44
:10FD500002460B46FEF77AFA00220023FEF754FD16
:10FD6000D9E600200021D6E60000E0FE422EE63F64
:10FD7000763C7935EF39EA3D44523EDF12F1C23F1D
:10FD8000DE03CB966446C73F599322942449D23F61
:10FD9000935555555555E53F9FC678D0099AC33FB1
:10FDA000AF788E1DC571CC3F04FA97999999D93FC8
:10FDB000555555555555D53F00005043FFFFEF7F32
:10FDC0000000F03F0000E03F000050C32046FEF777
:10FDD0008BFB0FA3D3E9002380468946FEF7EAFB9D
:10FDE0000DA3D3E9002304460D4640464946FEF7DD
:10FDF000E1FB9AE702460B4650465946FEF726FAC3
:10FE0000DDE90223FEF7D6FB14E700BFAFF3008065
:10FE10000000E0FE422EE63F763C7935EF39EA3DC0
:10FE20000020704700200149704700BF0000F87FA4
:10FE3000014B1868704700BF3001002064000000CB
:10FE4000C8000000900100002003000040060000F0
:10FE5000800C000000190000003200000064000067
:10FE600050C3000088130000008000000000000064
:10FE700000000000000000000101C8004008000070
:10FE800032035400720069006E0061006D00690069
:10FE9000630020005300740065007000700065006E
:10FEA0007200200044006500760069006300650070
:10FEB000200026035400720069006E0061006D008E
:10FEC000690063004D006F00740069006F006E00F0
:10FED0002000430074006C0004030904090243007D
:10FEE000020100C0320904000001020201000524E1
:10FEF000001001052401000104240202052406006B
:10FF000001070582030800FF09040100020A00003E
:10FF100000070503024000000705810240000012AF
:10FF2000011001020000403C2A0001012C010203E3
:10FF300001010101000100000001000000010000BA
:10FF400000000001000000000000000000000000B0
:10FF5000000101010000000000000000000001009D
:10FF6000000000000001010100010100010100008A
:10FF70000000000000000000000000000000000081
:10FF80000000000000000000000000000000000071
:10FF9000000000000000000000000001010100005E
:10FFA000010001010100000000000000000000004D
:10FFB0000002000000000000010000000001020338
:10FFC0000401020304060708090204060831323658
:10FFD00030563134340000006C6F670000000000C0
:04FFE000F8B500BFB1
:04FFE400F8B500BFAD
:08FFE800B8F1FF7F01000000E9
:10FFF000CDFF000800010000000102000008000021
:020000040801F1
:1000000001000000020000000000000000000000ED
:1000100000000000000000000000000000000000E0
:1000200000000000000000000000000000000000D0
:10003000000000000000000000C2010000000800F5
:1000400071900008658E0008758D0008898D000884
:100050008B8D0008E98D00080D8E0008418F000887
:100060004D8F0008598F000800000000400000007C
:100070001FFF000812000000DCFE00084300000023
:10008000D8FE000804000000B2FE000826000000B0
:1000900080FE000832000000140100201A00000059
:1000A000010000004DD90008518D00084DD900080D
:1000B0004DD900084DD900084DD900084DD9000888
:1000C0004DD90008698D0008040100004DD90008D1
:1000D0004DD90008398E00084DD900084DD90008C7
:1000E0004DD900084DD90008458D00084DD90008AC
:1000F0004DD900084DD900084DD900084DD9000848
:100100004DD900081A0354004D0043005300540019
:10011000450050000000000000000000000000004A
:10012000380100200000000000000000240400202E
:100130008C040020F40400200000000000000000F7
:1001400000000000000000000000000000000000AF
:10015000000000000000000000000000000000009F
:10016000000000000000000000000000000000008F
:10017000000000000000000000000000000000007F
:10018000000000000000000000000000000000006F
:10019000000000000000000000000000000000005F
:1001A000000000000000000000000000000000004F
:1001B000000000000000000000000000000000003F
:1001C000000000000000000000000000000000002F
:1001D00001000000000000000E33CDAB34126DE6CC
:1001E000ECDE05000B000000000000000000000035
:1001F00000000000000000000000000000000000FF
:1002000000000000000000000000000000000000EE
:1002100000000000000000000000000000000000DE
:1002200000000000000000000000000000000000CE
:0405500001000000A6
:04000005080041109E
:00000001FF
